:107689000000090200000301FA0400EF0500030AE3
:107699000A5A0B001E0C00FA0D00030E00040F011C
:1076A90064100096120132130AFA14010217010A32
:1076B9001801EF1905321A010A1B01EF1C05321FC7
:1076C900FFFF20FFFF23011E2400642A00FA2B007C
:1076D900FA2C50782D003D2E004630006432507847
:1076E9003300003432FA3501643601643701503809
:1076F9000A643A00033B00043C00643E003C3F003E
:107709000140FFFF411450420A5A430AC844053256
:107719004500B44600FA4900024B00014C00FA50FA
:107729000606510596520A32530B46540A965705D6
:1077390046590A465A32FA5B010A5C0A325E000A65
:107749005F00646200FE64021067FFFF680101695F
:1077590001016A05966B00006C32966D0004730096
:10776900017400017801327901327E00648100647C
:1077790084FFFF8800028A00019D0A969E00019FEE
:10778900FFFFA00124A2000AA3FFFFA4FFFFA5FF9A
:10779900FFA6FFFFA7FFFFA8FFFFA9FFFF01014801
:1077A9001500022F003C4701484802045601044EC7
:1077B900FFFF58000261FFFF6600028500AF8600E7
:1077C900018700FA890109990006A100FAFAFAFA73
:1077D9000101241500022F1E3C47014848020456A6
:1077E90001034EFFFF58000261FFFF66000285009A
:1077F900AF8600018700FA890109990000A10000FC
:10780900FAFAFA0101241500002F1E3C4701244809
:1078190002035601014EFFFF58000061FFFF660099
:107829000085FFFF86FFFF87FFFF8901029900009E
:10783900A10000FAFAFA0065006F00790083008D53
:10784900009700A100AC00B600C000CA00D400DE59
:1078590000E800F2005800600068007000780080BD
:1078690000880090009800A000A800B000B800C1EE
:1078790000C800D000D800DF00E600EE00F60041A5
:107889000047004D00530059005F0065006C00710E
:107899000077007D00830089008F0095009B00A27E
:1078A90000A700AC00B200B900C000C500CA00D2F0
:0A78B90000D500DD00E100E700EF5C
:103CD80075A71085F97485FA757E017F00E5751260
:103CE80079D5E5742FFF50010E8E5A8F5B9000181E
:103CF800E0FCA3E0FDEF2DFDEE3CFC8C5C8D5D90BF
:103D08000038E0FAA3E0FBED2BFBEC3AFA8A5C8B77
:103D18005D2275A71085F97485FA757E017F00E527
:103D2800751279D5E5742FFF50010E8E5A8F5BAC52
:103D38002DAD2EEF2DFDEE3CFC8C5C8D5D9000389A
:103D4800E0FAA3E0FBED2BFBEC3AFA8A5C8B5D22F0
:103D5800E55DF5FBE55CF5FCD29322E55DF5E9E56B
:103D68005CF5EAD29422E55DF5EBE55CF5ECD291E1
:103D780022E55DF5EDE55CF5EED29222E55DF5FD17
:103D8800E55CF5FED28722E55DF5CEE55CF5CFD2A0
:103D98009022A203B34008E5B54480F5B58006E556
:103DA800B5547FF5B522123CD89008F3E0B402026E
:103DB8008003023ED8A220B35003023E489001225D
:103DC800E0D3950C4024900018E0FEA3E0FFE50C3A
:103DD80090011A127A06E01279D574C88E048F05FC
:103DE800FF1279C58C5C8D5D800A900018E0F55C47
:103DF800A3E0F55DAE5CAF5D745E1279D574058E97
:103E0800048F05FF1279C5AE5AAF5BED2FFFEC3E6C
:103E1800FE8E5C8F5D900038E0FCA3E0FDEF2DFD89
:103E2800EE3CFC8C5C8D5DE50C90708FF828287357
:0D3E3800123D588008123D638003123D6E5C
:09708F00023E38023E3D023E4281
:103E4500023ECC900122E0FEE50C2403C39E5024E3
:103E5500900018E0FEA3E0FFE50C90011D127A0624
:103E6500E01279D574C88E048F05FF1279C58C5C74
:103E75008D5D800A900018E0F55CA3E0F55DAE5C11
:103E8500AF5D745E1279D574058E048F05FF1279C6
:103E9500C5AE5AAF5BED2FFFEC3EFE8E5C8F5D909D
:103EA5000038E0FCA3E0FDEF2DFDEE3CFC8C5C8DC5
:103EB5005DE50C907098F8282873123D79800812FA
:073EC5003D848003123D8FD4
:09709800023EBF023EC4023EC9E3
:103ECC009000EFE0B40103123D9A8029E50C90704C
:103EDC00A1F8282873123D58123D79800E123D63CB
:0B3EEC00123D848006123D6E123D84E2
:0970A100023EE1023EE9023EF16B
:103EF7009000EFE0B40103123D9A22123CD8E50C82
:103F07009070AAF8282873123D58802E123D6390AE
:103F170000EFE0C394025006A203B3B3400280024D
:103F2700D2878016123D6E9000EFE0C394025006D0
:0A3F3700A203B3B340028002D2904F
:0970AA00023F0E023F13023F2BCE
:103F41009000D1E0B4031FE50C9070B3F8282873FA
:0A3F5100D2928006D2878002D2903F
:0970B300023F51023F55023F5912
:103F5B009000EFE0B40103123D9A80429000EFE035
:103F6B00B40219123D1AE50C9070BCF82828731294
:0C3F7B003D798008123D848003123D8FC8
:0970BC00023F7A023F7F023F848B
:103F87009000EFE0B40106A203B3B340028013E54B
:103F97000C9070C5F8282873D2928006D2878002C9
:023FA700D290B6
:0970C500023F9F023FA3023FA716
:103FA90022E50C9070CEF8282873024046A23CB353
:103FB9004008E5B54408F5B58006E5B554F7F5B50B
:103FC900807BA23CB34008E5B54402F5B58006E51F
:103FD900B554FDF5B58066A23CB34008E5B544107B
:103FE900F5B58006E5B554EFF5B58051A23CB3406F
:103FF90008E5B54420F5B58006E5B554DFF5B5808B
:104009003CA23CB34008E5B54440F5B58006E5B5AA
:1040190054BFF5B58027A23CB34008E5B54480F507
:10402900B58006E5B5547FF5B58012A23C92928021
:0D4039000CA23C92878006A23C9290800071
:1070CE00023FB3023FB6023FCB023FE0023FF50262
:1070DE00400A02401F02403402403A024040024041
:0170EE00465B
:10404600227453900160F07475900161F07462906F
:104056000162F07461900163F07472900164F0740F
:1040660075900165F07420900166F07436900167D2
:10407600F07443900168F07479900169F0746C9063
:10408600016AF0742090016BF0743390016CF07447
:104096003690016DF0745490016EF022900897E00E
:1040A600FEA3E0FF741DD39F74019E400C90768999
:1040B600120048E493F599804C90F802E493B40515
:1040C60014900897E0FEA3E0FF9076BC120048E447
:1040D60093F599803090F802E493D39405401490B8
:1040E6000897E0FEA3E0FF907689120048E493F576
:1040F600998012900897E0FEA3E0FF9076EF1200F9
:1041060048E493F5999008971279E3900897E0FEB2
:10411600A3E0FFEFB45007EEB40103754E0022AEE4
:104126005AAF5B740A8E048F05FF1279C58C5C8DBD
:104136005DAE5AAF5B740A8E048F05FF1279F08C60
:104146005A8D5BC200E55B455A6013740AC3955BE2
:10415600FFE4955AFE8E5A8F5B785C127A28E574D6
:10416600A85CB80015D3955D4010E574C3955DFF56
:10417600E4955CFE8E5C8F5D8012E5742424C39505
:104186005DFFE4955CFE8E5C8F5DD200757400AEBB
:104196005CAF5D740B6F4E6006740C6F4E7018AE9C
:1041A6005CAF5D740B6F4E7005757401800375749A
:1041B60002755D0A755C00AE5CAF5D740E6F4E6095
:1041C60006740F6F4E7018AE5CAF5D740E6F4E7056
:1041D600057574018003757402755D0D755C00AE1E
:1041E6005CAF5D74236F4E600674246F4E7018AE1C
:1041F6005CAF5D74236F4E70057574018003757432
:1042060002755D22755C002290009DE0B40104C237
:10421600078002D20790009EE0B40104C208800223
:10422600D2089000DBE075F0E1A4FFAEF0740A8ED0
:10423600048F05FF1279C590088BECF0A3EDF09082
:1042460000DBE075F02BA4FFAEF0900014EEF0A3B7
:10425600EFF07E017F00900099E01279D59000DCA6
:10426600E08E048F05FF1279C5740AFF1279C58D99
:10427600619000E5E075F0E1A4FFAEF0740A8E04EB
:104286008F05FF1279C590088FECF0A3EDF0900032
:10429600E7E060139000E7E0F5F0741684FF7E0017
:1042A600EF9008EDF0800674649008EDF09000DD64
:1042B600E0900077F0900129E0900084F090012BC7
:1042C600E0FE9000D9E08E0088F0A4FFAEF0EF90FB
:1042D60008F6F0900104E075F013A4FDACF0900030
:1042E60038ECF0A3EDF0A225B34016900175E0700E
:1042F6000C900176E07006900177E060028002C2C1
:1043060025900175E0B4300F900176E0B44708902F
:104316000177E0643B60028004D2268002C22674E4
:10432600E3900076F09000C6E0B40B0874E39000CA
:1043360076F0805A9000C6E0B419129000DCE09046
:10434600782A12008CE493900076F080419000C6A3
:10435600E0B41E129000DCE090784812008CE493E2
:10436600900076F080289000C6E0B428129000DC19
:10437600E090787212008CE493900076F0800F90B3
:1043860000C6E0B446089000BDE0900076F09000CC
:1043960096E0FE9008F7E06E601B7599E612019CA8
:1043A60074AB900050F012069A7464F50975080013
:1043B6001205E480FE90008EE0700674009000C343
:1043C600F090007BE0FE9000C3E0B5066390007EAF
:1043D600E0FE9000E1E0B5065790007CE0FE90001C
:1043E600EFE0B5064B900082E0FE900096E0B50641
:1043F6003F90007FE0FE9000D1E0B5063390007D4F
:10440600E0FE9000DFE0B50627900080E0FE900019
:10441600FCE0B5061B900081E0FE9000FDE0B506CD
:104426000F900083E0FE90010FE06E70030246DEFF
:1044360090009EE070089000DFE064046002800651
:1044460074039000DFF0900058E0C39405500874A0
:1044560002900112F0801D9000D1E0D39402500624
:104466009000EFE060087406900112F0800674096F
:10447600900112F0900096E0B40106740090009648
:10448600F0900096E0B4020674009000E1F090000F
:1044960096E0B4030674009000EEF09000E1E0D3DD
:1044A60094014026741B900114F074009000AAF049
:1044B60074009006DFF074009006E0F09000C3E010
:1044C600600674009000C3F080329000C3E0601A6A
:1044D6007400900114F0741B9000AAF0740090060A
:1044E600DFF074009006E0F080127400900114F082
:1044F60074009000AAF0741B9006DFF09000D1E0E3
:10450600D3940240089000EFE064026002800674D3
:10451600009000EFF09000D1E0D3940240089000A4
:10452600EFE0640160028027741C900115F07400AE
:104536009000ABF074009006E3F074009006E4F08F
:104546009000C3E0B4020674019000C3F08033907B
:1045560000C3E0B4021A7400900115F0741C9000B8
:10456600ABF074009006E3F074009006E4F080125D
:104576007400900115F074009000ABF0741C900666
:10458600E3F09000FCE060147407900116F07400EC
:104596009006D7F074009006D8F0800C7400900155
:1045A60016F074079006D7F09000FDE060147408CA
:1045B600900117F074009006DBF074009006DCF0B2
:1045C600800C7400900117F074089006DBF09001DF
:1045D6000FE06014742A900787F074009006D3F0F9
:1045E60074009006D4F0800C7400900787F0742A4B
:1045F6009006D3F09000D1E0B402069000EFE060A0
:1046060002802674049006E7F074059006EBF074B9
:10461600069006EFF07400900782F074009007830E
:10462600F07400900784F0803674009006E7F0740A
:10463600009006E8F074009006EBF074009006EC2B
:10464600F074009006EFF074009006F0F074049099
:104656000782F07405900783F07406900784F09043
:1046660000DFE0D394024014741890077AF07419AE
:1046760090077BF0741A90077CF080127400900704
:104686007AF0740090077BF0740090077CF0D224D7
:104696009000C3E090007BF09000EFE090007CF08B
:1046A6009000E1E090007EF09000D1E090007FF075
:1046B6009000DFE090007DF0900096E0900082F0A0
:1046C6009000FCE0900080F09000FDE0900081F00A
:1046D60090010FE0900083F09000F9E0B40117908C
:1046E6000024740FF0A374FFF0900026E4F0A3F00A
:1046F60074029000F9F09000F9E0B40341900026AE
:10470600E0FEA3E0FF900024E0FCA3E0FD127A2087
:1047160074101279D57408120039EF9000F8F0EF92
:10472600700674FF9000F8F074009000F9F09000A5
:1047360025E09000AFF0900024E09000B0F09000EB
:104746008AE0900087F0900089E0900086F0900063
:10475600B8E0C3941E50569000B8E0F404241E90AE
:104766000088F0900088E075F00A84FF7E008F7460
:10477600900088E075F00A84ADF07C008D7590009D
:1047860086E0D39575400D900086E0C39575900040
:1047960086F0800F900086E0240AC3957590008607
:1047A600F00574900087E02574900087F0900087EC
:1047B600E0900046F0900046E0240C900047F09010
:1047C6000046E02418900048F0900046E0D3944854
:1047D600400B900046E0C39448900046F090004796
:1047E600E0D39448400B900047E0C39448900047BC
:1047F600F0900048E0D39448400B900048E0C39402
:1048060048900048F0C228900046E0D39424400D1A
:10481600900046E0C39424900046F0D228C2299026
:104826000047E0D39424400D900047E0C3942490C1
:104836000047F0D229C22A900048E0D39424400DC4
:10484600900048E0C39424900048F0D22A90004C8F
:10485600E4F0900046E0640B6007900046E0B40C7C
:1048660020900046E0B40B06740290004CF09000D5
:1048760046E0B40C0690004C7401F0740D900046AE
:10488600F0900046E0640E6007900046E0B40F200A
:10489600900046E0B40E06740290004CF09000467C
:1048A600E0B40F0690004C7401F07410900046F0CE
:1048B600900046E064236007900046E0B424209010
:1048C6000046E0B42306740290004CF0900046E0E7
:1048D600B4240690004C7401F09000467401F090E8
:1048E600004DE4F0900047E0640B6007900047E05D
:1048F600B40C20900047E0B40B06740290004DF013
:10490600900047E0B40C0690004D7401F0740D90D1
:104916000047F0900047E0640E6007900047E0B45F
:104926000F20900047E0B40E06740290004DF09000
:104936000047E0B40F0690004D7401F0741090002B
:1049460047F0900047E064236007900047E0B424F6
:1049560020900047E0B42306740290004DF09000CA
:1049660047E0B4240690004D7401F09000477401AE
:10497600F090004EE4F0900048E0640B6007900071
:1049860048E0B40C20900048E0B40B067402900096
:104996004EF0900048E0B40C0690004E7401F0749E
:1049A6000D900048F0900048E0640E6007900048C3
:1049B600E0B40F20900048E0B40E06740290004E5A
:1049C600F0900048E0B40F0690004E7401F07410A9
:1049D600900048F0900048E064236007900048E0AB
:1049E600B42420900048E0B42306740290004EF0F0
:1049F600900048E0B4240690004E7401F090004800
:104A06007401F090008AE0FE9000EDE02E900051D7
:104A1600F0900051E0D39424400B900051E0C394F1
:104A260024900051F0900051E0D39424400B900064
:104A360051E0C39424900051F09000C8E0B4010204
:104A46008003024B14900051E09070EFF828287311
:104A5600024AEE024AEE024AEE024AEE024AEE022C
:104A66004AEE024AEE024AEE807E807C807A740A22
:104A7600900051F08072740D900051F0806A806849
:104A8600740D900051F080607410900051F08058C1
:104A96008056805480527412900051F0804A7415EA
:104AA600900051F080428040803E803C803A8038C1
:104AB6008036741A900051F0802E741D900051F0CB
:104AC60080268024741D900051F0801C7420900074
:104AD60051F0801480128010800E7422900051F0E4
:084AE60080069000517401F0FC
:1070EF00024A56024A59024A5C024A5F024A620247
:1070FF004A65024A68024A6B024A6E024A70024AA5
:10710F0072024A74024A7C024A84024A86024A8EFA
:10711F00024A96024A98024A9A024A9C024AA402DA
:10712F004AAC024AAE024AB0024AB2024AB4024A1A
:10713F00B6024AB8024AC0024AC8024ACA024AD232
:0F714F00024ADA024ADC024ADE024AE0024AE859
:104AEE00900051E0D39412400D900051E0C3941207
:104AFE00900052F0800A900051E02412900052F083
:104B0E00755E12024BC9900051E090715EF8282834
:104B1E0073024BB2024BB29000517401F0024BB2D1
:104B2E007404900051F0807C807A80788076807456
:104B3E0080728070806E740A900051F08066740DE1
:104B4E00900051F0805E805C740D900051F08054A6
:104B5E007410900051F0804C804A8048804680440A
:104B6E0080428040803E7416900051F08036741959
:104B7E00900051F0802E802C7419900051F08024FA
:104B8E00741C900051F0801C801A801880168014BE
:104B9E0080128010800E7422900051F080069000DA
:044BAE00517401F04D
:10715E00024B1F024B22024B25024B2E024B3602D4
:10716E004B38024B3A024B3C024B3E024B40024B19
:10717E0042024B44024B4C024B54024B56024B5EA6
:10718E00024B66024B68024B6A024B6C024B6E025C
:10719E004B70024B72024B74024B7C024B84024BBF
:1071AE0086024B8E024B96024B98024B9A024B9CD8
:0F71BE00024B9E024BA0024BA2024BA4024BAC11
:104BB200900051E0D3940C400B900051E0C3940C50
:104BC200900051F0755E0C90008AE0FE9000D0E0FB
:104BD200D39E501390008AE0FE9000D0E0F4042EA1
:104BE20004900049F0801390008AE02448FE90006F
:104BF200D0E0F4042E04900049F0900049E0D394F0
:104C020024400F900049E0C39424900049F0D21F41
:104C12008002C21F900049E09071CDF828287302EB
:104C22004CB6024CB69000497401F0024CB67404C2
:104C3200900049F0807E807C807A807880768074D3
:104C420080728070740A900049F08068740D900040
:104C520049F08060805E740D900049F080567410B7
:104C6200900049F0804E804C804A804880468044C3
:104C7200804280407416900049F080387419900088
:104C820049F08030802E7419900049F08026741CFF
:104C9200900049F0801E801C801A801880168014B3
:104CA200801280107422900049F0800890004974AC
:044CB20001F0B21F3C
:1071CD00024C21024C24024C27024C30024C380256
:1071DD004C3A024C3C024C3E024C40024C42024C9A
:1071ED0044024C46024C4E024C56024C58024C6026
:1071FD00024C68024C6A024C6C024C6E024C7002DE
:10720D004C72024C74024C76024C7E024C86024C3F
:10721D0088024C90024C98024C9A024C9C024C9E57
:0F722D00024CA0024CA2024CA4024CA6024CAE92
:104CB600900049E0240C90004AF0900049E0241846
:104CC60090004BF090004AE0D39424400B90004AA9
:104CD600E0C3942490004AF090004BE0D394244023
:104CE6000B90004BE0C3942490004BF012019C22E1
:104CF600C293C294C291C292C287C290E5B554EFE4
:104D0600F5B5E5B554DFF5B5C296C295C2A0C29712
:104D1600C2A2C2A1E5B554BFF5B5E5B5547FF5B558
:104D2600E5B554FBF5B5C209755F469000D3E07052
:104D360005756E028003756E0375550075540090F7
:104D4600000C74FFF0A374DCF0C20FC212C215741B
:104D5600C890003AF074C890003EF074C8900042C3
:104D6600F0755300755200C204754700E570B41320
:104D76000375700075640090001AE4F0A3F0757175
:104D860010C20CC20DC20EC20375570075560090B4
:104D9600000EE4F0A3F0900010E4F0A3F0C22C752E
:104DA6005900755800900095E075F032A4FFAEF0FA
:104DB600900022EEF0A3EFF0900085E4F09008F367
:104DC600E4F0C227D21CC21BD21DC21EC21FC220C3
:104DD600900012E4F0A3F022755B00755A00AE5AFB
:104DE600AF5B741CC39F74019E5003024ED2907633
:104DF60089120048E493645F602390768912004824
:104E0600E493647E6017907689120048E493648187
:104E1600600B907689120048E493B48403024EB284
:104E2600AE5AAF5B907689120048E49390008912DF
:104E36007A060FBF00010EE0FC907689120048EC5E
:104E4600FEE493FFEEC39F5026AE5AAF5B0FBF0042
:104E5600010E907689120048AE5AAF5BE493FC903F
:104E66007689120048E493900089127A06ECF0AE37
:104E76005AAF5B907689120048E493900089127AC3
:104E860006E0FC90768B120048ECFCE493FDECD334
:104E96009D401990768B120048E493FC9076891217
:104EA6000048E493900089127A06ECF0AE5AAF5BA4
:104EB60074022FFF50010E8E5A8F5B785B740126A9
:104EC600F6500418E436F64003024DE422755B0002
:104ED600755A00AE5AAF5B7432BE00039F50030290
:104EE6004FA09077A6120048E493900089127A06A4
:104EF6000FBF00010EE0FC9077A6120048ECFEE41E
:104F060093FFEEC39F5026AE5AAF5B0FBF00010E54
:104F16009077A6120048AE5AAF5BE493FC9077A652
:104F2600120048E493900089127A06ECF0AE5AAF6C
:104F36005B9077A6120048E493900089127A06E007
:104F4600FC9077A8120048ECFCE493FDECD39D405E
:104F5600199077A8120048E493FC9077A6120048AF
:104F6600E493900089127A06ECF0AE5AAF5B742D8A
:104F76006F4E7006755B33755A00AE5AAF5B74029E
:104F86002FFF50010E8E5A8F5B785B740126F65008
:104F96000418E436F64003024ED922755B00755AB2
:104FA60000AE5AAF5B7432BE00039F500302506ED0
:104FB6009077D9120048E493900089127A060FBFC1
:104FC60000010EE0FC9077D9120048ECFEE493FF56
:104FD600EEC39F5026AE5AAF5B0FBF00010E90770F
:104FE600D9120048AE5AAF5BE493FC9077D9120011
:104FF60048E493900089127A06ECF0AE5AAF5B90C3
:1050060077D9120048E493900089127A06E0FC9062
:1050160077DB120048ECFCE493FDECD39D4019903D
:1050260077DB120048E493FC9077D9120048E493AA
:10503600900089127A06ECF0AE5AAF5B742D6F4E73
:105046007006755B33755A00AE5AAF5B74022FFF5C
:1050560050010E8E5A8F5B785B740126F650041849
:10506600E436F64003024FA722755B00755A00AE80
:105076005AAF5B7432BE00039F500302513C9078D6
:105086000C120048E493900089127A060FBF0001C3
:105096000EE0FC90780C120048ECFEE493FFEEC3A1
:1050A6009F5026AE5AAF5B0FBF00010E90780C12D0
:1050B6000048AE5AAF5BE493FC90780C120048E4CB
:1050C60093900089127A06ECF0AE5AAF5B90780C9A
:1050D600120048E493900089127A06E0FC90780E5C
:1050E600120048ECFCE493FDECD39D401990780E39
:1050F600120048E493FC90780C120048E493900068
:1051060089127A06ECF0AE5AAF5B742D6F4E7006BC
:10511600755B33755A00AE5AAF5B74022FFF5001B0
:105126000E8E5A8F5B785B740126F6500418E436AF
:10513600F640030250752275A71085F97485FA7535
:105146007E017F00E5751279D5E5742FFF50010EBB
:105156008E5A8F5BAC5CAD5DEF2DFDEE3CFC8C5C3E
:105166008D5D123D58123D63123D6E9000D1E0D325
:1051760094024009123D79123D84123D8F75A700B5
:105186002285F97485FA757E017F00E5751279D559
:10519600E5742FFF50010E8E5A8F5B7E017F76904D
:1051A600010EE01279D5AC5AAD5BED2FFFEC3EFE59
:1051B6008E5C8F5DE55DF5EDE55CF5EE900077E4E0
:1051C600F07412900054F02285F97485FA757E0108
:1051D6007F00E5751279D5E5742FFF50010E8E5AC2
:1051E6008F5B900014E0FCA3E0FDEF2DFDEE3CFC90
:1051F6008C5C8D5DE55DF5FDE55CF5FE22056522C1
:10520600A2DBB340089000DDE0900077F0A2DCB3AB
:105216004048A29650067419900054F0A295500684
:105226007419900054F0A2A050067419900054F01E
:10523600A29750067419900054F0A2A25006741951
:10524600900054F0A2A150067419900054F0C29632
:10525600C295C2A0C297C2A2C2A175D8402285A794
:105266007375A7109000D1E0D3940250079000EF19
:10527600E0B40252A2D8B34002C293A2D9B340020C
:10528600C294A2DAB34002C2919000D1E0640260F7
:10529600079000D1E0B40417A2DBB34002C292A289
:1052A600DCB34002C287A2DDB34002C2908015A2E1
:1052B600D8B34002C292A2D9B34002C287A2DAB3DF
:1052C6004002C290802DA2D8B3400AC2939000EF4C
:1052D600E06002C292A2D9B3400AC2949000EFE005
:1052E6006002C287A2DAB3400AC2919000EFE06082
:1052F60002C29075D8408573A72290F800E49364A3
:1053060006600280FE12009E75A70075D80075D94A
:105316000475DD0975DE0975D84075A71075D800C6
:1053260075D90475DA0975DB0975DC0975DD09754A
:10533600DE0975DF0975D84075A7001200FB74C831
:10534600F5097508001205E475A70FE5FC900063E2
:10535600F0E5FB900064F0E5FA900065F0E5F99061
:105366000066F075A70090F800E493F5281207038D
:105376009008A0E0D3940350079008A0E0B401067B
:1053860074009008A0F09008A0E09008F7F074016F
:105396009000D2F09008A0E090723CF82828738024
:1053A6002A802875A70F75F30F75A700A2A34006DC
:1053B60074029000D2F0801375A70F75F31775A7C6
:0B53C60000A2A4400674029000D2F088
:0C723C000253A50253A70253A90253BE3F
:1053D1009000D2E0B4022AC21A120AAC7402900000
:1053E100D2F09008A0E0907248F8282873801080CD
:0F53F1000E74009000E1F0800674009000EEF062
:0C7248000253EE0253F00253F20253FA1C
:105400008028D21A1209C174019000D2F09008A02D
:10541000E0907254F82828738010800E7400900079
:0A542000E1F0800674009000EEF049
:0C72540002541802541A02541C02542464
:10542A0090F807E493900070F0900070E0440890C0
:10543A000070F0900070E054FE900070F012039D2E
:10544A001240479008ADE0900175F09008AEE090E8
:10545A000176F09008AFE0900177F0900175E07066
:10546A000C900176E07006900177E060028004C239
:10547A00258002D2259000C3E00490007BF0124DF3
:10548A00DE90F802E493B40505124FA1801290F859
:10549A0002E493D394054005124ED3800312506F51
:1054AA0074009000F9F012420EE5B54401F5B574A6
:1054BA0006900056F07400900057F074019000585E
:1054CA00F090F802E493900059F090F803E4939076
:1054DA00005AF090F804E49390005BF07406900090
:1054EA005CF0900059E0B40506740590005CF090F9
:1054FA000059E0B40406740490005CF0742E900025
:10550A005DF0740390005EF0740690005FF074071B
:10551A00900060F090F805E493900061F090F8062E
:10552A00E493900062F0740090006AF074009000B6
:10553A006BF0740090006CF0740090006DF07400D1
:10554A0090006EF0740090006FF074FF900071F09C
:10555A00A2B6B39205A2B3B39206A2A4B39222A2B0
:10556A00A3B39223900072E4F0757000743A900726
:10557A0089F074FD90078AF0900073E4F0756F016A
:10558A00900054E4F09000D3E0B40106741A90003D
:10559A0054F0C221756400C20AD20BC203757200AC
:1055AA00C224120586756000756C00756200756606
:1055BA0032756700756800756900756A00756B0059
:1055CA0090001AE4F0A3F0756D00D2B2D2A4D2B062
:1055DA00D2B1D2A3D2A7D2A6D2A5D2B77E017F00DA
:1055EA009000B0E01279D59000AFE02FFF50010E85
:1055FA00900024EEF0A3EFF0EFD394FFEE940F4067
:10560A0007900024E4F0A3F09000F8E0700674FF1D
:10561A009000F8F09000D3E07005756E0280037573
:10562A006E037400900118F07400900119F0742947
:10563A009006CFF07415900777F07416900778F0FB
:10564A007417900779F0740090077DF07400900742
:10565A007EF0740190077FF07402900780F0740363
:10566A00900781F07400900785F07400900786F027
:10567A00D29CE571D3941040037571109006D0E066
:10568A00D3940C400674009006D0F09006D4E0D370
:10569A00940C400674009006D4F09006D8E0D39497
:1056AA000C400674009006D8F09006DCE0D3940C07
:1056BA00400674009006DCF09006E0E0D3940C40BB
:1056CA000674009006E0F09006E4E0D3940C4006DD
:1056DA0074009006E4F09006E8E0D3940C40067457
:1056EA00009006E8F09006ECE0D3940C40067400B3
:1056FA009006ECF09006F0E0D3940C40067400900B
:10570A0006F0F0D2EC75CF01A298B34005C2981208
:10571A000C14E54E6006A299B3B340028005C29903
:10572A001210A3E54F64016005E54FB4040280D569
:10573A00C28E7E107F00E5651279D5E58D75F01071
:10574A00A4FDACF0EF2DFDEE3CFCE58B75F010846A
:10575A00FF7E00ED2FFFEC3EFE8E548F55D28E90C9
:10576A0000B6E060099000B6E0C3943D400280565E
:10577A0090001C1279E390001CE0FEA3E0FF900069
:10578A001EE0FCA3E0FDEFB5053CEEB50438B21807
:10579A00A204B34013A218B34008E5B54404F5B512
:1057AA008006E5B554FBF5B590001EE0FEA3E0FFC8
:1057BA00900020E0FCA3E0FDEF2DFDEE3CFC900004
:1057CA001EECF0A3EDF09000C3E060099000C3E086
:1057DA00C394034003025887122FCEA204400890B4
:1057EA0000ADE0F546801BE560C39561500575463E
:1057FA0000800F90009AE0C3956250069000C0E0C6
:10580A00F546E54675F002A4FFAEF0900895EEF075
:10581A00A3EFF0AC2FAD30EDD39FEC9E402CE5B555
:10582A0054BFF5B59006D0E07006E5B554F7F5B566
:10583A009000C3E0B402099000E1E0C39402400280
:10584A008006E5B54480F5B58033900072E0C394D4
:10585A0041502AE5B54440F5B59006D0E07006E51A
:10586A00B54408F5B59000C3E0B402099000E1E040
:10587A00C3940240028006E5B5547FF5B59000C393
:10588A00E0B403241230E9AE2FAF30900895E0FC63
:10589A00A3E0FDEFD39DEE9C4008E5B54440F5B585
:1058AA008006E5B554BFF5B590009EE06009A2B345
:1058BA00300601B3B340028056A2B3300601B340AA
:1058CA004EA2B3300801B34039A21C403090008484
:1058DA00E0D3955F40259008F3E07013900085E0CF
:1058EA00B401069008F37401F0900085E004F0A278
:1058FA001BB34005900085E4F0D21BD21CA208B36A
:10590A009206A208B330B301B34004A2089206A2D9
:10591A00B6300501B35003026086A2B6300501B362
:10592A005003026086A2B6300701B35003025FA497
:10593A00756F009000B6E0B43D13A207B34008E5C6
:10594A00B554FBF5B58006E5B54404F5B5055FA287
:10595A0009B3B35013AE54AF5590000CE0FCA3E06A
:10596A00FDEDC39FEC9E4003025B45E55FB40B0669
:10597A00755F0D025B28E56EB4032EA22CB340229C
:10598A00E55FB42303756E01E55FC3942350069067
:10599A0000547401F0E55FD394234006740290002A
:1059AA0054F0755F01D22C8066E56EB4020A756EFA
:1059BA0001755F23C21BC21DE55FB42305755F0134
:1059CA00804D900054E07038E55FC39423500690F0
:1059DA0000547401F0E55FD39423400674029000EA
:1059EA0054F0E55FC394235002D221E55FD3942398
:1059FA004002D221C296C295C2A0C297C2A2C2A137
:105A0A009000D3E0B40105124CF68003755F019053
:105A1A0000B6E060099000B6E0C3943D40028043BE
:105A2A0090001CE0FEA3E0FF9000B6E08E048F0514
:105A3A00FF1279C574018C068D0712003990002077
:105A4A00EEF0A3EFF0900020E0F8A3E090001EC86B
:105A5A00F0A3C8F090001CE4F0A3F0C218E5B55416
:105A6A00FBF5B5A2A4B34002C222A2A3B34002C26C
:105A7A0023A221B34002C221B21E9008F3E0B4016E
:105A8A0011A21BB34004D21E8002C21E74029008E7
:105A9A00F3F09008F3E0C394025006A204B3B340B3
:105AAA0002800674029008F3F09000DFE06404605C
:105ABA00079000D1E0B4046290009EE0600690086E
:105ACA00F3E07002800DA21D301B01B34005900067
:105ADA0085E4F09000D3E064016006A227B3B350D6
:105AEA001790009EE06009A21B301D01B3B340026B
:105AFA0080067405900054F0B21DA21CB3401BA28C
:105B0A001BB34004D21D8002C21D9000D3E0700670
:105B1A009008F3E070028002D227C21BC21CAE5664
:105B2A00AF57AC54AD55EF2DFDEE3CFC74028C061C
:105B3A008D071200398E568F57805CE55FB40E1DB3
:105B4A00AE56AF57AC54AD55EF2DFDEE3CFC74028A
:105B5A008C068D071200398E568F57801BAE56AFB2
:105B6A0057AC54AD55EF2DFDEE3CFC74018C068DFF
:105B7A00071200398E568F57E56EC39402500DAE48
:105B8A0054AF557498C39F743A9E40028009124CD0
:105B9A00F67406900054F0E55FB40E03755F10E5E5
:105BAA005FB423127403900054F0D2219000D3E022
:105BBA00B40103124CF6AE58AF59AC54AD55EF2DA3
:105BCA00FDEE3CFC8C588D59AE54AF55EFD39DEE8B
:105BDA009C4011900012E0FAA3E0FBEBC394E8EAC0
:105BEA009403400280069000121279E3900010E0BC
:105BFA00FEA3E0FFAC54AD55EF2DFDEE3CFC90004A
:105C0A0010ECF0A3EDF09000D3E0B40118AE54AF5D
:105C1A005574051279D5740112003990000CEEF012
:105C2A00A3EFF08011AE54AF5574021279D59000EB
:105C3A000CEEF0A3EFF0C28E758D00758B007565C2
:105C4A0000755501755400D28EE55F240875F00978
:105C5A0084AFF07E00EF4E6003025CE8E56E6013ED
:105C6A00AE56AF5774091279D590000EEEF0A3EF35
:105C7A00F0800F900010E0F8A3E090000EC8F0A3A7
:105C8A00C8F090000EE0FEA3E0FFEF4E600B7C7CB4
:105C9A007D311278C38E528F53900010E4F0A3F036
:105CAA00AE52AF537428BE00039F5010E5642FFF15
:105CBA0050010E74011200398E528F53855364902D
:105CCA0000DAE0A852B8000DD395534008E5539086
:105CDA000053F080099000DAE014900053F090002D
:105CEA00D1E0B40408900049E0655F6002800EA22A
:105CFA001E301F01B34004D2208002C220E55F6437
:105D0A000A6005E55FB41C099000C3E06003122C29
:105D1A00849000C8E0B40114900051E0655F600708
:105D2A00900052E0B55F03757000801E900051E04C
:105D3A00655F6013900051E0240C655F6009900074
:105D4A0051E02418B55F03757000A20A5003025E81
:105D5A00C79000DFE0C394045006A209B3B340031E
:105D6A00025E1290008FE0B40173900111E0B40258
:105D7A0014121244900078E075F0BCA4FFAEF08EC5
:105D8A005C8F5D8056E56875F00A84FF7E00900599
:105D9A0089120048E0F55B755A00AE5AAF5B900075
:105DAA00B4E01279D574648E048F05FF1279C58C1C
:105DBA005C8D5DE55D90004FF0AE5AAF5B90008D53
:105DCA00E01279D574648E048F05FF1279C574BC0C
:105DDA008C068D071279D58E5C8F5D801790008DA9
:105DEA00E075F0BCA4FFAEF08E5C8F5D9000B4E06D
:105DFA0090004FF0E562C394CC5006E55D455C70B7
:105E0A0002800312513DD20A9000DFE0B4040690EA
:105E1A0008F3E07003025EC790008FE0B40173904C
:105E2A000111E0B40214121244900078E075F0BC3B
:105E3A00A4FFAEF08E5C8F5D8056E56875F00A842B
:105E4A00FF7E00900589120048E0F55B755A00AEA6
:105E5A005AAF5B9000B4E01279D574648E048F0552
:105E6A00FF1279C58C5C8D5DE55D90004FF0AE5AEE
:105E7A00AF5B90008DE01279D574648E048F05FFB4
:105E8A001279C574BC8C068D071279D58E5C8F5D2C
:105E9A00801790008DE075F0BCA4FFAEF08E5C8F89
:105EAA005D9000B4E090004FF0E562C394CC5006D8
:105EBA00E55D455C7002800312513DD20AE56EB47D
:105ECA000106E55F6411600280189000DFE0B40407
:105EDA000575710380097571009000557401F0759C
:105EEA006E00E56E6003025F9F9000D6E0600D9041
:105EFA000077E0A852B8000695534002804090000F
:105F0A00D6E0B4021F900046E0655F600F9000473C
:105F1A00E0655F6007900048E0B55F03757103753F
:105F2A006D00800CC201756D0090001AE4F0A3F0B8
:105F3A00900077E060067409900054F08057900052
:105F4A0046E0655F600F900047E0655F600790007C
:105F5A0048E0B55F409000DFE0B4040FA227B340E9
:105F6A0005757100800375710380037571009000D7
:105F7A0046E0B55F069000557401F0900047E0B521
:105F8A005F067402900055F0900048E0B55F067411
:105F9A0003900055F0A207B39205A207B330B601E9
:105FAA00B35003026086756F019000B6E0B43D13EA
:105FBA00A207B34008E5B54404F5B58006E5B55433
:105FCA00FBF5B5E5B54401F5B5742B900072F0A266
:105FDA00079205E55FD3944A4014D209E55FD3944A
:105FEA006D400B7405900054F0D221755F46900005
:105FFA00DEE0B40107E56BC3944140028018E56B0B
:10600A00C3941450087413900054F08006740E90D0
:10601A000054F0124CF690005CE0FE900059E0C388
:10602A009E4009900059E0D39408400974FB9000FF
:10603A0054F0124CF690005AE0601590005AE0FEB7
:10604A00900058E06E600974FC900054F0124CF60F
:10605A0090005BE0601590005BE0FE90005DE06EF2
:10606A00600974FE900054F0124CF69008A0E060AB
:10607A000690010EE060028003120B97A221B34042
:10608A000CC296C295C2A0C297C2A2C2A190010E2A
:10609A00E0600CAE52AF537414BE00059F400280FC
:1060AA0037900096E0907260F8282873802A80283A
:1060BA00A2A3B35005A223B340028005125187D28E
:1060CA00238015A2A4B35005A222B3400280051270
:0860DA005187D22280028000F0
:107260000260B60260B80260BA0260CD0260E0025D
:0272700060E2DA
:1060E200A20CB3B35008900049E0655F6002802DB6
:1060F200A202B35006A201B3B34002801A9000D1AB
:10610200E0B404097400F50C123DAE80077400F58A
:106112000C123F0275A700C20CD20DD20EA20DB313
:10612200B3500890004AE0655F6002802DA202B37E
:106132005006A201B3B34002801A9000D1E0B40429
:10614200097401F50C123DAE80077401F50C123F83
:106152000275A700D20CC20DD20EA20EB3B3500824
:1061620090004BE0655F6002802DA202B35006A250
:1061720001B3B34002801A9000D1E0B40409740262
:10618200F50C123DAE80077402F50C123F0275A7A2
:1061920000D20CD20DC20EE571907272F8282873EB
:0461A2009000F6E093
:037272000261A214
:1061A6009072FFF82828731225CF80121225CF800F
:0E61B6000D12265980081227058003122705B6
:0F72FF000261AD0261B20261B70261BC0261C1FE
:1061C4007571010266FD12283112294875710202A7
:1061D40066FD122CC8A204B340139000DBE075F0F6
:1061E4001DA4FFAEF0900014EEF0A3EFF090088928
:1061F400E0FEA3E0FF740A1279D590000EE0FCA340
:10620400E0FD74098F02FF1279C58D078C038E049B
:106214008A058B061278C390088DEEF0A3EFF090F8
:1062240000DFE0B401087450BE00059F4002800DF9
:10623400745090088DF8E4F0E8A3F0801B90088D6A
:10624400E0FEA3E0FF74F0BE00039F500B74F090D7
:10625400088DF8E4F0E8A3F0E53770037537019092
:10626400088DE0FEA3E0FFE5372FFF50010E9008F4
:106274008DEEF0A3EFF0757103A233401A90005530
:01628400E039
:067275000261CA0261D6AD
:1062850090730EF8282873800D75710A8008757152
:066295000B800375710C83
:0C730E0002628C02628E0262930262989E
:10629B000266FD9006D0E060077401F508122DF63A
:1062AB00A235B3B35008900787E0642A60028009D7
:1062BB00E5B54402F5B50263659000C4E0D39402E2
:1062CB004045900098E02403A852B8000495535021
:1062DB000990009AE0D395625002800ED202A22B55
:1062EB0040067408900054F0D22B900098E0A8520E
:1062FB00B80005D39553500B90009AE02403C39537
:10630B00625002C2028053900098E02403A852B856
:10631B00000495535010E560C39561500990009AA5
:10632B00E0D395625002800ED202A22B4006740875
:10633B00900054F0D22B900098E0A852B80005D3EF
:10634B0095535014E561240FC39560400B90009A50
:10635B00E02403C395625002C202A2024002C22B88
:10636B00A235B3500DA202B35008900787E0642A00
:10637B0060028006E5B554FDF5B59000DEE07007D0
:10638B00E56BC3941440028002D2029000D3E0B4B8
:10639B000102D202A2024005757104800A757110C8
:0E63AB0090001AE4F0A3F00266FD9000C4E03A
:06727B0002629E0263B5F1
:1063B90090731AF828287312135A801212135A80EC
:0E63C9000D12150D80081215C480031215C4A4
:0F731A000263C00263C50263CA0263CF0263D479
:1063D7009006D4E060077402F508122DF675710572
:1063E7000266FD12171D7571069006D8E0600774E6
:1063F70003F508122DF69006DCE060077404F50833
:10640700122DF60266FD90004FE06006A204B3B3BA
:106417004002800DE55FD3940C500690004FE014C6
:10642700F01219A67571079006E0E060077405F58C
:1064370008122DF69006E4E060077406F508122DA1
:10644700F60266FD900111E0B402031212CB121E90
:106457000E7571089006E8E060077407F508122DBD
:10646700F69006ECE060077408F508122DF6026650
:10647700FD121EF07571090266FD1222C8A20CB347
:106487005005A20DB340028006D20CD20DD20E7574
:1064970071109006F0E060077409F508122DF602F6
:1064A70066FD90003CE0C39446500AC296C29774BA
:1064B7004690003CF090004CE0B4011DE537240AFB
:1064C700F53790088DE0FEA3E0FF740A2FFF500117
:1064D7000E90088DEEF0A3EFF090004CE0B4021D93
:1064E700E5372414F53790088DE0FEA3E0FF741418
:1064F7002FFF50010E90088DEEF0A3EFF085375B6C
:10650700755A00900046E0F574124125E55D90004C
:106517003CF0900006E55AF0A3E55BF0E5749000C7
:106527003DF0C21090088DE0F55AA3E0F55B9000AE
:1065370046E0F574124125E55D90003AF0900000C1
:10654700E55AF0A3E55BF0E57490003BF0A20092FA
:106557001190004CE06002B211C20F757103026620
:10656700FD900040E0C3944650139000DFE0B40173
:1065770002C296C295C2A27446900040F090004DA8
:10658700E0B4011DE537240AF53790088DE0FEA336
:10659700E0FF740A2FFF50010E90088DEEF0A3EF75
:1065A700F090004DE0B4021DE5372414F53790084C
:1065B7008DE0FEA3E0FF74142FFF50010E90088DAD
:1065C700EEF0A3EFF085375B755A00900047E0F5D2
:1065D70074124125E55D900040F0900008E55AF0FF
:1065E700A3E55BF0E574900041F0C21390088DE0DD
:1065F700F55AA3E0F55B900047E0F574124125E5F5
:106607005D90003EF0900002E55AF0A3E55BF0E5EF
:106617007490003FF0A200921490004DE06002B227
:1066270014C2127571030266FD900044E0C39446DC
:1066370050139000DFE0B40102C296C2A0C2A17459
:1066470046900044F090004EE0B4011DE537240A5F
:10665700F53790088DE0FEA3E0FF740A2FFF500185
:106667000E90088DEEF0A3EFF090004EE0B4021DFF
:10667700E5372414F53790088DE0FEA3E0FF741486
:106687002FFF50010E90088DEEF0A3EFF085375BDA
:10669700755A00900048E0F574124125E55D9000B9
:1066A70044F090000AE55AF0A3E55BF0E57490002A
:1066B70045F0C21690088DE0F55AA3E0F55B90000F
:1066C70048E0F574124125E55D900042F090000422
:1066D700E55AF0A3E55BF0E574900043F0A2009261
:1066E7001790004EE06002B217C21575710380065D
:0666F70080048002800017
:107281000263EA02640D02644B02647802648102C3
:1072910064A90265680266300266F70266F9026651
:0472A100FB0266FD89
:1066FD0090003AE0B55F0280030267DAA20F4072A4
:10670D00900000E0FEA3E0FFEF4E6021AE56AF57C4
:10671D00900000E0FCA3E0FD120003740A8E048FCC
:10672D0005FF1279C5900000ECF0A3EDF090003B51
:10673D00E0601A900000E0FEA3E0FFAC56AD57EF0D
:10674D002DFDEE3CFC900000ECF0A3EDF090003B35
:10675D00E0D39401401A900000E0FEA3E0FFAC5698
:10676D00AD57EF2DFDEE3CFC900000ECF0A3EDF0ED
:10677D00D20FAE54AF55900000E0FCA3E0FDEFC387
:10678D009DEE9C40481251CE9000DFE09072A5F82E
:10679D002828738030D296802CD2968028D296D21B
:1067AD00978022A2114010A228301D01B34004D2BF
:1067BD00978002D296800EA228301D01B34004D2DC
:0567CD00968002D29746
:0F72A5000267A00267A20267A60267AA0267B08B
:1067D200C20F74C890003AF0A20FB3B350079000F2
:1067E2003AE0B55F0280481251CE9000DFE090722D
:1067F200B4F82828738030D296802CD2968028D282
:1068020096D2978022A2114010A228301D01B340D7
:1068120004D2978002D296800EA228301D01B34086
:0768220004D2968002D29718
:0F72B4000267F70267F90267FD026801026807C7
:1068290074C890003AF0C20F90003CE0B55F028056
:10683900030268D2A2104072900006E0FEA3E0FFB6
:10684900EF4E6021AE56AF57900006E0FCA3E0FD85
:10685900120003740A8E048F05FF1279C590000691
:10686900ECF0A3EDF090003DE0601A900006E0FE28
:10687900A3E0FFAC56AD57EF2DFDEE3CFC900006B2
:10688900ECF0A3EDF090003DE0D39401401A9000A4
:1068990006E0FEA3E0FFAC56AD57EF2DFDEE3CFC44
:1068A900900006ECF0A3EDF0D210AE54AF55900075
:1068B90006E0FCA3E0FDEFC39DEE9C400CC296C22E
:1068C90097744690003CF0C210A210B3B3500790E1
:1068D900003CE0B55F02800CC296C29774469000F6
:1068E9003CF0C21090003EE0B55F0280030269CA25
:1068F900A2124072900002E0FEA3E0FFEF4E602179
:10690900AE56AF57900002E0FCA3E0FD12000374FD
:106919000A8E048F05FF1279C5900002ECF0A3EDF1
:10692900F090003FE0601A900002E0FEA3E0FFACA7
:1069390056AD57EF2DFDEE3CFC900002ECF0A3EDB7
:10694900F090003FE0D39401401A900002E0FEA3CA
:10695900E0FFAC56AD57EF2DFDEE3CFC900002EC8C
:10696900F0A3EDF0D212AE54AF55900002E0FCA3B3
:10697900E0FDEFC39DEE9C40481251CE9000DFE050
:106989009072C3F82828738030D296802CD29580D3
:1069990028D295D2A28022A2144010A229301D012A
:1069A900B34004D2A28002D295800EA229301D01E3
:0969B900B34004D2958002D2A281
:0F72C30002699002699202699602699A0269A0B3
:1069C200C21274C890003EF0A212B3B350079000F6
:1069D2003EE0B55F0280481251CE9000DFE0907237
:1069E200D2F82828738030D296802CD2958028D273
:1069F20095D2A28022A2144010A229301D01B340D8
:106A020004D2A28002D295800EA229301D01B34089
:076A120004D2958002D2A21C
:0F72D2000269E70269E90269ED0269F10269F7F1
:106A190074C890003EF0C212900040E0B55F028059
:106A290003026ACBA2134072900008E0FEA3E0FFC4
:106A3900EF4E6021AE56AF57900008E0FCA3E0FD91
:106A4900120003740A8E048F05FF1279C59000089D
:106A5900ECF0A3EDF0900041E0601A900008E0FE30
:106A6900A3E0FFAC56AD57EF2DFDEE3CFC900008BE
:106A7900ECF0A3EDF0900041E0D39401401A9000AE
:106A890008E0FEA3E0FFAC56AD57EF2DFDEE3CFC50
:106A9900900008ECF0A3EDF0D213AE54AF5590007E
:106AA90008E0FCA3E0FDEFC39DEE9C40159000DFDC
:106AB900E0B40102C296C295C2A27446900040F0A9
:106AC900C213A213B3B35007900040E0B55F028030
:106AD900159000DFE0B40102C296C295C2A27446C5
:106AE900900040F0C213900042E0B55F02800302BB
:106AF9006BCCA2154072900004E0FEA3E0FFEF4EBC
:106B09006021AE56AF57900004E0FCA3E0FD1200EF
:106B190003740A8E048F05FF1279C5900004ECF006
:106B2900A3EDF0900043E0601A900004E0FEA3E0BA
:106B3900FFAC56AD57EF2DFDEE3CFC900004ECF098
:106B4900A3EDF0900043E0D39401401A900004E0D3
:106B5900FEA3E0FFAC56AD57EF2DFDEE3CFC9000D7
:106B690004ECF0A3EDF0D215AE54AF55900004E05B
:106B7900FCA3E0FDEFC39DEE9C40481251CE90006E
:106B8900DFE09072E1F82828738030D296802CD209
:106B9900A08028D2A0D2A18022A2174010A22A3018
:106BA9001D01B34004D2A18002D2A0800EA22A30D6
:0B6BB9001D01B34004D2A08002D2A155
:0F72E100026B92026B94026B98026B9C026BA281
:106BC400C21574C8900042F0A215B3B350079000E8
:106BD40042E0B55F0280481251CE9000DFE090722F
:106BE400F0F82828738030D296802CD2A08028D246
:106BF400A0D2A18022A2174010A22A301D01B340C6
:106C040004D2A18002D2A0800EA22A301D01B3407A
:076C140004D2A08002D2A10E
:0F72F000026BE9026BEB026BEF026BF3026BF9BF
:106C1B0074C8900042F0C215900044E0B55F02804A
:106C2B0003026CCDA216407290000AE0FEA3E0FFB7
:106C3B00EF4E6021AE56AF5790000AE0FCA3E0FD8B
:106C4B00120003740A8E048F05FF1279C590000A97
:106C5B00ECF0A3EDF0900045E0601A90000AE0FE26
:106C6B00A3E0FFAC56AD57EF2DFDEE3CFC90000AB8
:106C7B00ECF0A3EDF0900045E0D39401401A9000A6
:106C8B000AE0FEA3E0FFAC56AD57EF2DFDEE3CFC4A
:106C9B0090000AECF0A3EDF0D216AE54AF55900075
:106CAB000AE0FCA3E0FDEFC39DEE9C40159000DFD6
:106CBB00E0B40102C296C2A0C2A17446900044F097
:106CCB00C216A216B3B35007900044E0B55F028022
:106CDB00159000DFE0B40102C296C2A0C2A17446B7
:106CEB00900044F0C2169000E1E0B402028003026F
:106CFB006E19900074E0D395675064900074E0F4C3
:106D0B00042567FE9000E4E08E00F5F0E884FF7E3A
:106D1B00008F74EFC39410500CEF8574F0A4FDAC8E
:106D2B00F08D7480037574FF900074E0D3957440FC
:106D3B000B900074E0C39574F5728003757200902C
:106D4B0000FFE0D3957240069000FFE0F5729001D2
:106D5B0000E0C395725006900100E0F572807190CF
:106D6B000074E0C39567FE9000E4E08E00F5F0E858
:106D7B0084FF7E008F74EFC39410500CEF8574F07A
:106D8B00A4FDACF08D7480037574FF85745B755A2C
:106D9B0000900074E0255BFFAE5A50010E8E5A8FA7
:106DAB005B74FFBE0009D39F4005855B7280037542
:106DBB0072FF9000FFE0D3957240069000FFE0F564
:106DCB0072900100E0C395725006900100E0F572DD
:106DDB00A204B3B3500D900075E0FE9000ECE0D32D
:106DEB009E5002800E7407900054F0E5B554BFF529
:106DFB00B5801B75A710E5CDC395724008E5B5545A
:106E0B00BFF5B58006E5B54440F5B575A700900014
:106E1B00FCE0605E900106E0A852B8000495535068
:106E2B0017900105E0A852B8000ED3955340099076
:106E3B000107E0D395624002801D75A710E5CDC315
:106E4B0094BF4008E5B554EFF5B58006E5B54410A1
:106E5B00F5B575A700801B75A710E5CDC394404011
:106E6B0008E5B554EFF5B58006E5B54410F5B575F5
:106E7B00A7009000FDE0605E900109E0A852B80009
:106E8B000495535017900108E0A852B8000ED39503
:106E9B0053400990010AE0D395624002801D75A70B
:106EAB0010E5CDC394BF4008E5B554DFF5B58006BA
:106EBB00E5B54420F5B575A700801B75A710E5CD8A
:106ECB00C394404008E5B554DFF5B58006E5B544FD
:106EDB0020F5B575A700E570C39413501DE57075CB
:106EEB00F00284AFF07E00EF4E7005123290800AF4
:106EFB00A2EDB34005C2ED123290AE54AF5574986B
:106F0B00C39F743A9E400C900073E0C3945A4003A5
:106F1B0002708CA209B34009124CF674069000540F
:106F2B00F0A20BB3500EE562D394334007E562C376
:106F3B0094CC40028041900111E0B402141212442F
:106F4B00900078E075F05EA4FFAEF08E5C8F5D80F4
:106F5B000F90008DE075F05EA4FFAEF08E5C8F5D40
:106F6B00E55D455C6011E5B54401F5B5742B90000A
:106F7B0072F012513DD20B900073E0D39401400795
:106F8B00E562C3941A40028002C20B9006D0E06007
:106F9B00077401F508122DF69006D4E06007740211
:106FAB00F508122DF69006D8E060077403F5081269
:106FBB002DF69006DCE060077404F508122DF690B0
:106FCB0006E0E060077405F508122DF69006E4E084
:106FDB0060077406F508122DF69006E8E06007745A
:106FEB0007F508122DF69006ECE060077408F5081B
:106FFB00122DF69006F0E060077409F508122DF6D5
:10700B00900073E0C3945A5010E570B413099000CC
:10701B0073E004F0757000803FE570B41303757076
:10702B0000C28E758D00758B0075650075550175E9
:10703B005400D28E900072E0C394415008900072BD
:10704B00E004F080067441900072F0900072E0B49E
:10705B004106E5B554FEF5B5900073E0D3940140BD
:10706B0007E56BC3944140028006740E900054F008
:10707B009008A0E0600690010EE060028003120B06
:04708B009702570F02
:107329000000010001400160018001A001C001E0ED
:1073390002000300039603B603D603F40400050014
:107349000512052405360548055A056C057E059084
:1073590005A805C005DE0600061406280646066EC1
:1073690006AE05CF06EE00FF013F015F017F019FD9
:1073790001BF01DF01FF02FF039503B503D503F345
:1073890003FF04FF05110523053505470559056B5D
:10739900057D058F05A705BF05CE05F1061306274F
:1073A9000645066D06AD06ED05DD06FF0FAA0FA51C
:1073B9000F9F0F9A0F940F8D0F870F800F780F7102
:1073C9000F680F600F570F4E0F450F3B0F300F25FA
:1073D9000F1A0F0E0F020EF50EE80EDB0ECC0EBEC5
:1073E9000EAE0E9F0E8E0E7D0E6C0E5A0E470E348B
:1073F9000E200E0C0DF70DE20DCB0DB50D9D0D8573
:107409000D6D0D540D3A0D200D050CE90CCE0CB186
:107419000C940C760C580C3A0C1B0BFB0BDB0BBBBE
:107429000B9A0B790B570B350B130AF10ACE0AABE2
:107439000A870A640A400A1C09F809D409B0098CA8
:1074490009670943091F08FB08D608B2088E086AAC
:107459000846082307FF07DC07B907960773075192
:10746900072F070D06EC06CA06AA0689066906490A
:10747900062A060A05EC05CD05B0059205750558DD
:10748900053C0520050504EA04CF04B5049C0482E3
:107499000469045104390422040B03F403DE03C80C
:1074A90003B2039D038903750361034D033B03285D
:1074B9000316030402F202E102D102C002B002A0E3
:1074C900029102820273026502570249023C022FAD
:1074D90002220216020901FD01F201E601DB01D0D7
:1074E90001C601BB01B101A7019D0194018B018274
:1074F9000179017001680160015801500148014199
:1075090001390132012B0125011E01180111010B5D
:10751900010500FF00FA0FA60FA00F990F920F8B1C
:107529000F840F7C0F740F6B0F620F580F4E0F43B0
:107539000F380F2C0F1F0F120F050EF70EE80ED87C
:107549000EC80EB70EA50E930E800E6C0E580E4285
:107559000E2C0E150DFD0DE40DCB0DB10D950D790C
:107569000D5D0D3F0D200D010CE10CC00C9E0C7C36
:107579000C590C350C100BEA0BC40B9E0B760B4FF8
:107589000B260AFD0AD40AAA0A800A550A2A09FF03
:1075990009D409A8097C0950092508F908CD08A1C9
:1075A9000875084A081E07F307C8079D07730749A6
:1075B900072006F706CE06A6067E06570630060AF7
:1075C90005E405BF059B057705540532051004EF51
:1075D90004CE04AE048F047104530435041903FD69
:1075E90003E203C703AD0394037B0363034B033433
:1075F900031E030802F302DE02CA02B602A30291C5
:10760900027F026D025C024C023C022C021D020E3A
:10761900020001F201E401D701CA01BE01B101A6CC
:10762900019A018F0185017A01700166015D01539B
:10763900014A0141013901310129012101190112CF
:10764900010B010400FD00F700F000EA00E400DE90
:1076590000D900D300CE00C900C400BF00BA00B5EC
:1076690000B100AD00A800A400A0009C00990095FD
:107679000091008E008A008700840081007E007BD3
:10009E0075B50075840175A70075FFA075EF069004
:1000AE000050E4F075C91075A70F75A1C775A700AC
:1000BE0075D90075CE0C75A70F75F1FE75F2FF752B
:1000CE00F30775F47875A4BA75A5FF75A60775AE16
:1000DE000075AFFF75D48175D5FF75D6FF75D7FF47
:1000EE0075A70075A20175A14775F8092275E60876
:1000FE0075E71075BC0175BE0475BD6C75BE0775D0
:10010E00BDA075BE0875BD0175BC0075BB1875BC6C
:10011E002075BA0875E88075D11375A70F75E105BE
:10012E0075E20075C740124CF6759700759780748E
:10013E000A1279B57597C0E5975420700280F8754C
:10014E008F0275A700D2AF75980075A90C75A70F11
:10015E0075AB4375ADFB75AC1E75A71075C91875DB
:10016E00CA0075CB0075C80475A700758912758E07
:10017E0004758C00758A00C2A9D28C758D00758BA2
:10018E0000D2ABD28E75B62075D944C2992290009A
:10019E008BE090089FF0900096E09008A0F0900001
:1001AE0097E09008A1F09000B6E09008A2F09000C1
:1001BE00C3E09008A3F09000D1E09008A4F0900066
:1001CE00DFE09008A5F09000E1E09008A6F0900026
:1001DE00EFE09008A7F09000FCE09008A8F09000E7
:1001EE00FDE09008A9F090010FE09008AAF09001B0
:1001FE0027E09008ACF0900175E09008ADF090010A
:10020E0076E09008AEF0900177E09008AFF09001A4
:10021E000EE09008B0F09000F8E09008B1F0900079
:10022E00AFE09008B2F09000B0E09008B3F090000C
:10023E00AAE09008B4F09000ABE09008B5F0900101
:10024E0014E09008B6F0900115E09008B7F0900118
:10025E0016E09008B8F0900117E09008B9F0900100
:10026E0018E09008BAF09006CFE09008BBF0900628
:10027E00D3E09008BCF09006D7E09008BDF0900651
:10028E00DBE09008BEF09006DFE09008BFF090062D
:10029E00E3E09008C0F09006E7E09008C1F0900609
:1002AE00EBE09008C2F09006EFE09008C3F09006E5
:1002BE00F3E09008C4F0900777E09008C5F090073F
:1002CE0078E09008C6F0900779E09008C7F09007A4
:1002DE007AE09008C8F090077BE09008C9F090078C
:1002EE007CE09008CAF090077DE09008CBF0900774
:1002FE007EE09008CCF090077FE09008CDF090075C
:10030E0080E09008CEF0900781E09008CFF0900743
:10031E0082E09008D0F0900783E09008D1F090072B
:10032E0084E09008D2F0900785E09008D3F0900713
:10033E0086E09008D4F0900787E09008D5F0900101
:10034E0019E09008D6F090011AE09008D7F09001CD
:10035E001BE09008D8F090011CE09008D9F09001B5
:10036E001DE09008DAF090011EE09008DBF090019D
:10037E001FE09008DCF0900120E09008DDF0900185
:10038E0021E09008DEF0900122E09008DFF022904C
:10039E00089FE090008BF09008A0E0900096F090FF
:1003AE0008A1E0900097F09008A2E09000B6F090BF
:1003BE0008A3E09000C3F09008A4E09000D1F09064
:1003CE0008A5E09000DFF09008A6E09000E1F09024
:1003DE0008A7E09000EFF09008A8E09000FCF090E5
:1003EE0008A9E09000FDF09008AAE090010FF090AF
:1003FE0008ACE0900127F09008B0E090010EF0906C
:10040E0008B1E09000F8F09008B2E09000AFF090E4
:10041E0008B3E09000B0F09008B4E09000AAF0901D
:10042E0008B5E09000ABF09008B6E0900114F090A3
:10043E0008B7E0900115F09008B8E0900116F09022
:10044E0008B9E0900117F09008BAE0900118F0900A
:10045E0008BBE09006CFF09008BCE09006D3F09079
:10046E0008BDE09006D7F09008BEE09006DBF09055
:10047E0008BFE09006DFF09008C0E09006E3F09031
:10048E0008C1E09006E7F09008C2E09006EBF0900D
:10049E0008C3E09006EFF09008C4E09006F3F090E9
:1004AE0008C5E0900777F09008C6E0900778F090C6
:1004BE0008C7E0900779F09008C8E090077AF090AE
:1004CE0008C9E090077BF09008CAE090077CF09096
:1004DE0008CBE090077DF09008CCE090077EF0907E
:1004EE0008CDE090077FF09008CEE0900780F09066
:1004FE0008CFE0900781F09008D0E0900782F0904E
:10050E0008D1E0900783F09008D2E0900784F09035
:10051E0008D3E0900785F09008D4E0900786F0901D
:10052E0008D5E0900787F09008D6E0900119F0907A
:10053E0008D7E090011AF09008D8E090011BF090D7
:10054E0008D9E090011CF09008DAE090011DF090BF
:10055E0008DBE090011EF09008DCE090011FF090A7
:10056E0008DDE0900120F09008DEE0900121F0908F
:10057E0008DFE0900122F022754800900897E4F021
:10058E00A3F0753200753100754E00754F00C22F05
:10059E00D2309008A0E06002D22474FE900899F840
:1005AE00E4F0E8A3F074FE90089DF8E4F0E8A3F000
:1005BE0074FE90089BF8E4F0E8A3F0745A9008F1EA
:1005CE00F0745A9008F2F0D231C22DC233C232C248
:1005DE002EC235C23B22750B00750A00AE0AAF0B58
:1005EE00AC08AD09EDC39FEC9E401674FF1279B5B1
:1005FE0075CF01780B740126F6500418E436F650C8
:10060E00DB22C2AF75D904758F0375B7A575B7F127
:10061E0090F800E4F0758F0175B7A575B7F1E52870
:10062E0090F800F075B7A575B7F190F801E4F07584
:10063E00B7A575B7F19008E5E090F802F075B7A58B
:10064E0075B7F19008E9E090F803F075B7A575B7A6
:10065E00F19008E6E090F804F075B7A575B7F19043
:10066E0008E7E090F805F075B7A575B7F19008E8C2
:10067E00E090F806F075B7A575B7F19008EAE0902E
:10068E00F807F0758F0075D944D2AF22900050E074
:10069E00B4AB61C2AF75D90475B62275F522758FEC
:1006AE000375B7A575B7F1740090F600F0758F015C
:1006BE00755B00755A00AE5AAF5B7445BE00279F3E
:1006CE00402475B7A575B7F190089F120048E0FC5D
:1006DE0090F600120048ECF0785B740126F6500498
:1006EE0018E436F650D0758F0075F51175B6207575
:1006FE00D944D2AF22C2AF75F52275D904755B000D
:10070E00755A00AE5AAF5B7445BE00229F401F90D3
:10071E00F600120048E493FC90089F120048ECF09B
:10072E00785B740126F6500418E436F650D575D968
:10073E004475F511D2AF22900050E0B4AA028003A6
:10074E00020882C2AF75D90475B62275F522758F6F
:10075E000375B7A575B7F1740090F400F075B7A5E1
:10076E0075B7F1740090F200F075B7A575B7F17416
:10077E000090F000F075B7A575B7F1740090EE001B
:10078E00F0758F01755B00755A00AE5AAF5B74FF42
:10079E00C39F74019E402475B7A575B7F19000896B
:1007AE00120048E0FC90F400120048ECF0785B7404
:1007BE000126F6500418E436F650CF755B00755AD4
:1007CE0000AE5AAF5B74FFC39F74019E402475B791
:1007DE00A575B7F1900289120048E0FC90F2001264
:1007EE000048ECF0785B740126F6500418E436F6F7
:1007FE0050CF755B00755A00AE5AAF5B74FFC39F46
:10080E0074019E402475B7A575B7F1900489120046
:10081E0048E0FC90F000120048ECF0785B74012682
:10082E00F6500418E436F650CF755B00755A00AEDC
:10083E005AAF5B74FFC39F74019E402475B7A575B4
:10084E00B7F1900689120048E0FC90EE00120048C5
:10085E00ECF0785B740126F6500418E436F650CFAF
:10086E00758F0075F51175B62075D944D2AF743AEF
:10087E00900789F022900050E0B4AA02800302098A
:10088E00C0C2AF75D90475B62275F522758F037582
:10089E00B7A575B7F1740090EC00F075B7A575B7F4
:1008AE00F1740090EA00F075B7A575B7F174009079
:1008BE00E800F075B7A575B7F1740090E600F07515
:1008CE008F01755B00755A00AE5AAF5B74FFC39F04
:1008DE0074019E402475B7A575B7F190008912007A
:1008EE0048E0FC90EC00120048ECF0785B740126B6
:1008FE00F6500418E436F650CF755B00755A00AE0C
:10090E005AAF5B74FFC39F74019E402475B7A575E3
:10091E00B7F1900289120048E0FC90EA00120048FC
:10092E00ECF0785B740126F6500418E436F650CFDE
:10093E00755B00755A00AE5AAF5B74FFC39F7401AE
:10094E009E402475B7A575B7F1900489120048E052
:10095E00FC90E800120048ECF0785B740126F6502B
:10096E000418E436F650CF755B00755A00AE5AAFD8
:10097E005B74FFC39F74019E402475B7A575B7F1D4
:10098E00900689120048E0FC90E600120048ECF058
:10099E00785B740126F6500418E436F650CF758F46
:1009AE000075F51175B62075D944D2AF743A90071B
:1009BE0089F022C2AF75D90475F522755B00755AA0
:1009CE0000AE5AAF5B74FFC39F74019E401F90F43C
:1009DE0000120048E493FC900089120048ECF07875
:1009EE005B740126F6500418E436F650D4755B009D
:1009FE00755A00AE5AAF5B74FFC39F74019E401FC1
:100A0E0090F200120048E493FC900289120048EC28
:100A1E00F0785B740126F6500418E436F650D4755F
:100A2E005B00755A00AE5AAF5B74FFC39F74019E94
:100A3E00401F90F000120048E493FC9004891200CD
:100A4E0048ECF0785B740126F6500418E436F65044
:100A5E00D4755B00755A00AE5AAF5B74FFC39F74BA
:100A6E00019E401F90EE00120048E493FC90068910
:100A7E00120048ECF0785B740126F6500418E43648
:100A8E00F650D475F51175D944D2AF74019000D2D9
:100A9E00F0743A900789F09008F87401F022C2AF12
:100AAE0075D90475F522755B00755A00AE5AAF5BA9
:100ABE0074FFC39F74019E401F90EC00120048E427
:100ACE0093FC900089120048ECF0785B740126F6D6
:100ADE00500418E436F650D4755B00755A00AE5AC1
:100AEE00AF5B74FFC39F74019E401F90EA0012001B
:100AFE0048E493FC900289120048ECF0785B740194
:100B0E0026F6500418E436F650D4755B00755A007C
:100B1E00AE5AAF5B74FFC39F74019E401F90E800F6
:100B2E00120048E493FC900489120048ECF0785BC4
:100B3E00740126F6500418E436F650D4755B007531
:100B4E005A00AE5AAF5B74FFC39F74019E401F9054
:100B5E00E600120048E493FC900689120048ECF07F
:100B6E00785B740126F6500418E436F650D475F509
:100B7E001175D944D2AF74029000D2F0743A900736
:100B8E0089F074029008F8F02274019000D2F0906F
:100B9E0008A0E0903C1EF828287380188016A2A3A7
:100BAE00400674029000D2F0800AA2A4400674029D
:040BBE009000D2F0E1
:0C3C1E00020BA8020BAA020BAC020BB8B0
:100BC2009000D2E0B40105A239B34002801AD239B2
:100BD200124CF61209C174019000D2F012039D1258
:100BE2004047741B900054F09000D2E0B40206A279
:100BF20039B3B34002801AC239124CF6120AAC74ED
:100C0200029000D2F012039D124047741B900054D0
:100C1200F022E54F64046006E59964FF60028031CA
:100C2200A22F4004D22F8027E54F600874E6254F9B
:100C3200900054F0E54E600874F0254E900054F098
:100C4200E54FB4010280FE754F00754E00C22F8041
:100C520002C22FE54F903C2AF8282873754F00E511
:100C620099B4FF03754E01E599B4FE03754E02E592
:100C720099B4FD03754E03E599B4FC03754E04E582
:100C820099B4FA03754E05E599B4FB06754F011246
:100C92004CF6E599B4F906754F04124CF6E599B491
:100CA200F733124CF6C29C74AB900050F012069AC5
:100CB20074AA900050F09008F8E0B40105120745BC
:100CC2008003120883900050E4F0D29C754F0075A7
:100CD2004E007599F7E599D394E54007E599C394D9
:100CE200F040028016859950754F027E017F00E523
:100CF20050C394E61279D58E338F34900897E4F07E
:100D0200A3F0E599D394C24007E599C394E6400263
:100D12008028859950754F0374E5C39550F5347555
:100D22003300AE33AF349073291279A4E493F8748C
:100D32000193900897C8F0A3C8F0D2990210A2902C
:100D420008ACE0700AA225B35005A226B340028087
:100D52005C900897E0FEA3E0FF74FFBE00039F5083
:100D620009EFC39446EE9406402B900897E0FEA349
:100D7200E0FFEFD3946DEE94064009EFC394EEEEDC
:100D820094064011900897E0FEA3E0FFEFD394FF92
:100D9200EE94064013900897E0FEA3E0FF900089CE
:100DA200120048E599F080038599758011900897A3
:100DB200E0FEA3E0FF900089120048E599F0900858
:100DC200971279E3900897E0FEA3E0FFEFB40106E3
:100DD200EEB407028003020E9B900789E0B43C0246
:100DE2008003020E9BA225B35005A226B3400280C7
:100DF20055C29C12039D900096E09008F7F01242B3
:100E02000E900175E09008ADF0900176E09008AE8A
:100E1200F0900177E09008AFF074AB900050F012C0
:100E2200069A74AA900050F09008F8E0B4010512F6
:100E3200074580031208839008F8E09000D2F090F2
:100E42000050E4F08048C29C12019C74009008ADEE
:100E5200F074009008AEF074009008AFF090009625
:100E6200E09008F7F012420E74AB900050F01206B8
:100E72009A74AA900050F0120745120883D29C750A
:100E820099FB7464F5097508001205E480FED29C92
:100E9200754F00754E007599FB0210A2900897E0FD
:100EA200FEA3E0FFEF4E700685993275310090087F
:100EB20097E0FEA3E0FF74016F4E701BAC31AD32C0
:100EC200AA33AB34ED2BFBEC3AFA8A068B0790007F
:100ED20089120048E599F09008971279E3900897F3
:100EE200E0FEA3E0FF74026F4E7021AC31AD3274AC
:100EF200566D4C7006E55064E660028003124CF6B3
:100F020012420E855099754F00754E000210A29044
:100F12000897E0FEA3E0FF900089120048E599F0EF
:100F22009008971279E3900897E0FEA3E0FFAC33B4
:100F3200AD348F028E038C068D0790736F1279A4E5
:100F4200E493F9740193FEEAD39EEB99400985502C
:100F520099754F00754E000210A2900897E0FEA30B
:100F6200E0FF900089120048E599F0900897127905
:100F7200E3900897E0FEA3E0FFEFB40006EEB401B1
:100F82000280030210A2900066E0D394C7400B9047
:100F92000066E0C394C8F551801A900066E0D394CD
:100FA20063400B900066E0C39464F55180069000A4
:100FB20066E0F551E55175F002A4FFAEF08F74EFD3
:100FC200900089127A06EFFCE0FDEC90008C127A18
:100FD20006EDFCE0FDEC2DB5510280030210930FEB
:100FE200EF900089127A06E574FFE0FCEF90008D25
:100FF200127A06ECFFE0FCEFC39CB55102800302BB
:101002001093E57490008B127A06E574FFE0FCEF12
:1010120090008E127A06ECFFE0FCEF2CB55172E5DF
:101022007490008F127A06E0C395519008E5F0E5BE
:1010320074900090127A06E0C395519008E6F0E5AC
:1010420074900093127A06E0C395519008E7F0E598
:1010520074900094127A06E0C395519008E8F0E586
:1010620074900095127A06E0C395519008E9F0E574
:1010720074900096127A06E0C395519008EAF01235
:1010820006107599F97464F5097508001205E48073
:10109200FE7599FF7464F5097508001205E480FE77
:0F3C2A00020C5E020D41020E9E020F11020F5C92
:1010A20022E54E903C39F828287302118790089760
:1010B200E0FEA3E0FF900056120048E0F599900888
:1010C200971279E3900897E0FEA3E0FF741C6F4E3D
:1010D2007003754E00021187856F9902118790087F
:1010E20097E0FEA3E0FF900089120048E0F599EF37
:1010F200B40107EEB40703754E009008971279E326
:07110200021187900898E03C
:0F3C39000210AC0210AF0210DA0210E002110507
:10110900903CABF82828738553998067856099804E
:1011190062856299805D8566998058856899805352
:10112900856999804E856A998049856B9980449033
:10113900001BE0F599803CA230B340077599FAC2CB
:10114900308017A224B3400575990F800B90005485
:10115900E0F599900054E4F0C2248017856C9980D9
:1011690012856799800D856D9980087599FC8003B2
:03117900754E00B0
:103CAB0002111002111502111A02111F0211240226
:103CBB00112902112E021133021138021140021187
:0D3CCB006502116A02116F02117402117975
:0B117C009008971279E380031240A254
:033C4800021184E2
:1011870022E538255BFFAE5A50010E900089120008
:1011970048E0F539E538255BFFAE5A50010E0FBF21
:1011A70000010E900089120048E0F53A85403CE5C1
:1011B70039B53A058539388041E53AD39539401D27
:1011C700E53AC39539853BF0A4FFAEF0E53C8E04C4
:1011D7008F05FF1279C5ED2539F538801DE539C32F
:1011E700953A853BF0A4FFAEF0E53C8E048F05FFF2
:1011F7001279C5EDF4042539F53822E53AD3953946
:10120700401DE53AC39539853BF0A4FFAEF0E53CB8
:101217008E048F05FF1279C5ED2539F538801DE558
:1012270039C3953A853BF0A4FFAEF0E53C8E048FB9
:1012370005FF1279C5EDF4042539F5382290008FA2
:10124700E0B4017FE56875F00A84FF7E008F38E51A
:101257006875F00A84ADF07C008D3B75400A755ABD
:1012670005755B24E538C394115005121188800673
:101277009005BEE0F538E538C394F05008E538909E
:101287000078F0800674EF900078F0E56875F00A52
:1012970084FF7E008F38E56875F00A84ADF07C0026
:1012A7008D3B75400A755A05755B5AE538C394112D
:1012B700500512118880069005F4E0F538E538905E
:1012C700004FF02290008FE0B4010280030213590F
:1012D700E56875F00A84FF7E008F38E56875F00AC7
:1012E70084ADF07C008D3B75400A755A05755B36F9
:1012F700E538C39411500512118880069005D0E097
:10130700F538E538C394F0500585384C8003754CA3
:10131700EFE56875F00A84FF7E008F38E56875F0A1
:101327000A84ADF07C008D3B75400A755A05755BE4
:1013370048E538C39411500512118880069005E2DC
:10134700E0F538E538C394F0500585384D800375CE
:101357004DEF22E56075F00484FF7E008F38E5606D
:1013670075F00484ADF07C008D3B754004755A011F
:10137700755B00E538C3943F5005121188800690CD
:1013870001C8E0F538E538900891F8E4F0E8A3F0F3
:10139700900053E075F020A4FFAEF09000DAE08EE5
:1013A700048F05FF1279C58D389000C2E0D3956090
:1013B70050030214659000E6E0D395604010ED906D
:1013C70001C9127A06E0F52C752B00021462900011
:1013D700B1E0D395604043E5389001C9127A06E041
:1013E700F539E5389001E9127A06E0F53A9000E61A
:1013F700E0F4042560F53B9000B1E0FE9000E6E0E4
:10140700F4042EF53CE539B53A05853938800312E1
:10141700120285382C752B008041E5389001E912BE
:101427007A06E0F539E538900209127A06E0F53ACE
:101437009000B1E0F4042560F53B9000C2E0FE9017
:1014470000B1E0F4042EF53CE539B53A05853938A5
:10145700800312120285382C752B0002150C9000A0
:10146700E9E0D395605011E538900249127A06E019
:10147700F52C752B0002150C9000B2E0D395605047
:1014870043E538900229127A06E0F539E5389002EB
:1014970049127A06E0F53A9000B2E0F4042560F5C7
:1014A7003B9000E9E0FE9000B2E0F4042EF53CE545
:1014B70039B53A05853938800312120285382C75FB
:1014C7002B008041E538900209127A06E0F539E5EC
:1014D70038900229127A06E0F53A9000C2E0F40447
:1014E7002560F53B9000B2E0FE9000C2E0F4042EC8
:1014F700F53CE539B53A058539388003121202857E
:10150700382C752B00229000FAE0F53D75401175D7
:101517005A02755B00AE52AF53E53D75F00FA4FD5F
:10152700ACF0EDD39FEC9E4021E53D8E048F05FF87
:101537001279C5ED75F010A4FFAEF0E56075F011F6
:1015470084FD7C00ED2FF53E800EE56075F011847B
:10155700FF7E00EF24F0F53E853E38E56075F0111B
:1015670084AFF07E008F3B12118885383FAE52AFB3
:10157700539000FAE075F00FA4FDACF0EDD39FECAB
:101587009E4028755A02755B10853E381211888572
:101597003F3985383AAE52AF53E53D8E048F05FF8C
:1015A7001279F08D3B853D3C121202E53890089187
:1015B700F8E4F0E8A3F0752C64752B00229000FA8C
:1015C700E0F53D754011755A02755B00AE52AF5399
:1015D700E53D75F00FA4FDACF0EDD39FEC9E4021E7
:1015E700E53D8E048F05FF1279C5ED75F010A4FF58
:1015F700AEF0E56275F01184FD7C00ED2FF53E80BD
:101607000EE56275F01184FF7E00EF24F0F53E854C
:101617003E38E56275F01184AFF07E008F3B121102
:101627008885383FAE52AF539000FAE075F00FA4AB
:10163700FDACF0EDD39FEC9E4028755A02755B1008
:10164700853E38121188853F3985383AAE52AF53F7
:10165700E53D8E048F05FF1279F08D3B853D3C12E9
:101667001202E538900891F8E4F0E8A3F0E56C6021
:1016770017E56CC394FE50109000EEE0B402099099
:1016870000DCE0D3940B5002801F900891E0FEA38A
:10169700E0FFE56C1279D574E78E048F05FF1279A8
:1016A700C5900891ECF0A3EDF09000C4E0B4045F9E
:1016B700E56075F00484FF7E008F38E56075F004FF
:1016C70084ADF07C008D3B754004755A01755B0055
:1016D700E538C3943F500512118880069001C8E091
:1016E700F538900891E0FEA3E0FFE5381279D5744C
:1016F700328E048F05FF1279C5900891E0FEA3E0B2
:10170700FFEF2DFDEE3CFC900891ECF0A3EDF0759A
:101717002C64752B002290008FE0B40146E56875B4
:10172700F00A84FF7E008F38E56875F00A84ADF013
:101737007C008D3B75400A755A05755B00E538C31B
:1017470094115005121188800690059AE0F538AE7D
:101757002BAF2CE5382FFF50010E7464127A188EC8
:101767002B8F2C900090E0B40146E56975F00A8450
:10177700FF7E008F38E56975F00A84ADF07C008D37
:101787003B75400A755A05755B6CE538C394115073
:10179700051211888006900606E0F538AE2BAF2CAF
:1017A700E5382FFF50010E7464127A188E2B8F2C98
:1017B70090009FE0B40249E56BC3944175F005843E
:1017C700FF7E008F38E56B75F00584ADF07C008DEA
:1017D7003B754005755A06755B00E538C394135091
:1017E70005121188800690069CE0F538AE2BAF2CC9
:1017F700E5382FFF50010E7464127A188E2B8F2C48
:101807009000E1E0B4020280030218BCE56075F0C5
:101817001584FF7E008F38E56075F01584ADF07C88
:10182700008D3B754015755A03755BF4E538C39415
:101837000B50051211888006900488E0F538E538CA
:1018470075F0FFA4FFAEF09000E2E08E048F05FF75
:101857001279C5ED900074F0E56775F078A4FFAED6
:10186700F074FF8E048F05FF1279C58C5A8D5B7457
:10187700028C068D071200398F38AC5AAD5B7404A1
:10188700FF1279F08D3B754004755A06755B28E5A4
:1018970038C3941D500512118880069006CEE0F5D6
:1018A70038AE2BAF2CE5382FFF50010E7464127A37
:1018B700188E2B8F2C90008EE0B4025DE56275F0D8
:1018C70064A4FFAEF074081200398E5C8F5D740556
:1018D7008E048F05FF1279C58D38AE5CAF5D740538
:1018E7008E048F05FF1279F08D3B754005755A05FB
:1018F700755BDEE538C39413500512118880069096
:10190700067AE0F538AE2BAF2CE5382FFF50010EE5
:101917007464127A188E2B8F2C9000D0E0707F9011
:101927000053E075F00A84FF7E008F38900053E083
:1019370075F00A84ADF07C008D3B75400A755A0539
:10194700755BC0E538C3940E500512118880069068
:101957000657E0F538E538900079F09000EFE0B4ED
:10196700023C900053E075F00A84FF7E008F3890A8
:101977000053E075F00A84ADF07C008D3B75400A9A
:10198700755A05755BCFE538C3940E50051211885B
:101997008006900666E0F538E53890007AF02290E8
:1019A7000097E0B401179008ECE0252CFFAE2B5010
:1019B700010E9000EBE0127A188E2B8F2C90010FFE
:1019C700E0B40114900110E0A852B80004955350F8
:1019D70007E560C39561400280139000B9E0252CAC
:1019E700FFAE2B50010E8E2B8F2C021E0D900097F1
:1019F700E0B40306A22DB3B3400280509008F6E08E
:101A070070109008EFE0C39405A852B800069553EC
:101A1700400280109000B9E0252CFFAE2B50010E3C
:101A27008E2B8F2C9008F6E0600D9008EFE0A852FF
:101A3700B800069553400280109000B9E0252CFFAE
:101A4700AE2B50010E8E2B8F2C021E0D900091E0B5
:101A5700B402028003021E0D900094E0602FE56837
:101A6700D394464028900012E0FEA3E0FF9000CFF9
:101A7700E075F003A4FDACF0EFD39DEE9C400E9013
:101A870000F3E0A852B80005D395535003021E0D8A
:101A97009000C4E0B403028003021C5585625B75A5
:101AA7005A0090009BE0A852B800049553500E903E
:101AB700009CE0A85AB80005D3955B5003021C525E
:101AC700E56275F002A4FFAEF074158E048F05FF72
:101AD7001279C58C068D07900619120048FEE0FFA3
:101AE700EE900093E0FEEF8E0088F0A4FFAEF07456
:101AF700648E048F05FF1279C58C5A8D5B90005355
:101B0700E075F018A4FFAEF09000DAE08E048F05C0
:101B1700FF1279C58C068D07900631120048AE5A20
:101B2700AF5BE01279D574648E048F05FF1279C517
:101B37008C5A8D5BE566A85AB80005D3955B5003B0
:101B4700021BC9E566C3955BFFE4955AFE8E5A8F63
:101B57005B7428BE00039F500C755B28755A007490
:101B67000D900054F0AE5AAF5B900094E01279D517
:101B770074288E048F05FF1279C58C5A8D5B9008E7
:101B870091E0FEA3E0FF740A8E048F05FF1279C56A
:101B97008D068C07AC5AAD5BCFCECF120003740A0B
:101BA7008E048F05FF1279C58C5A8D5B900891E0E2
:101BB700FEA3E0FF127A20900891EEF0A3EFF00267
:101BC7001C52E566A85AB80004955B507EAE5AAF22
:101BD7005BE566127A188E5A8F5B7428BE00039FE6
:101BE700500C755B28755A00740D900054F0AE5A6E
:101BF700AF5B900094E01279D574288E048F05FFAF
:101C07001279C58C5A8D5B900891E0FEA3E0FF74B2
:101C17000A8E048F05FF1279C58D068C07AC5AAD65
:101C27005BCFCECF120003740A8E048F05FF1279A3
:101C3700C58C5A8D5B900891E0FEA3E0FFEF2DFD68
:101C4700EE3CFC900891ECF0A3EDF0021E0D900025
:101C5700DCE08560F0A4FFAEF074051279D5740757
:101C67001200398E5A8F5B90009BE0A852B800048F
:101C77009553501290009CE075F002A4FDACF0EF74
:101C8700C39DEE9C4003021E0DE56075F00B84FFBB
:101C97007E00900619120048FEE0FFEE900093E0E8
:101CA700FEEF8E0088F0A4FFAEF074648E048F05FB
:101CB700FF1279C58C5A8D5B900053E075F018A41C
:101CC700FFAEF09000DAE08E048F05FF1279C58C25
:101CD700068D07900631120048AE5AAF5BE01279C5
:101CE700D574648E048F05FF1279C58C5A8D5BE518
:101CF70066A85AB80005D3955B5003021D84E566B4
:101D0700C3955BFFE4955AFE8E5A8F5B7428BE001D
:101D1700039F500C755B28755A00740D900054F0A2
:101D2700AE5AAF5B900094E01279D574288E048F79
:101D370005FF1279C58C5A8D5B900891E0FEA3E0F0
:101D4700FF740A8E048F05FF1279C58D068C07ACC8
:101D57005AAD5BCFCECF120003740A8E048F05FFF6
:101D67001279C58C5A8D5B900891E0FEA3E0FF12B3
:101D77007A20900891EEF0A3EFF0021E0DE566A819
:101D87005AB80004955B507EAE5AAF5BE566127A8F
:101D9700188E5A8F5B7428BE00039F500C755B2802
:101DA700755A00740D900054F0AE5AAF5B900094D2
:101DB700E01279D574288E048F05FF1279C58C5AE5
:101DC7008D5B900891E0FEA3E0FF740A8E048F05F7
:101DD700FF1279C58D068C07AC5AAD5BCFCECF12FB
:101DE7000003740A8E048F05FF1279C58C5A8D5B28
:101DF700900891E0FEA3E0FFEF2DFDEE3CFC90087C
:101E070091ECF0A3EDF0229000EFE0B4027BE560E7
:101E170075F00884FF7E008F38E56075F00884ADA3
:101E2700F07C008D3B754008755A01755BE0E5381D
:101E3700C3943F50051211888006900288E0F53858
:101E4700E538900893F8E4F0E8A3F0900893E0FEF3
:101E5700A3E0FFAC2BAD2C12000374648E048F0536
:101E6700FF1279C5900893ECF0A3EDF090008CE099
:101E77008C068D071279D574648E048F05FF12794D
:101E8700C5900893ECF0A3EDF0900891E0FEA3E075
:101E9700FFAC2BAD2C12000374648E048F05FF1268
:101EA70079C5900891ECF0A3EDF090008CE08C06DA
:101EB7008D071279D574648E048F05FF1279C5904A
:101EC7000891ECF0A3EDF0A204401DAE52AF53749D
:101ED70005BE00039F5002D204E562D394CC4008AC
:101EE700D2027411900054F0229000EEE0B4020880
:101EF7009000DCE0640B60028045900891E0FEA34F
:101F0700E0FFE56C1279D574E78E048F05FF12792F
:101F1700C5900891ECF0A3EDF09000EFE0B4021F3C
:101F2700900893E0FEA3E0FFE56C1279D574E78E85
:101F3700048F05FF1279C5900893ECF0A3EDF0909C
:101F470000AEE05402601B9000A5E0A852B8001252
:101F5700D39553400DA204B3B35007E562C3949AD7
:101F67004002805FAE35AF369000A3E075F002A463
:101F7700FDACF0EF2DFDEE3CFC74022DFD50010C85
:101F8700E562BC003ED39D403A754401A23440331C
:101F97009000A4E075F05EA4FDACF07405FF127923
:101FA700C58C5C8D5D12513D900891E0FEA3E0FF6A
:101FB7009000A4E02FFF50010E900891EEF0A3EFE0
:101FC700F0D234E562A835B8000495365002C23421
:101FD700856236753500E54470030220E6900101FD
:101FE700E0C3954450030220D8900111E0C3940246
:101FF7004003022082E56875F00A84FF7E009005A1
:1020070089120048E0F55B755A00AE5AAF5B900045
:10201700A4E01279D574648E048F05FF1279C58CFC
:102027005C8D5D900101E004C395448C068D071219
:1020370079D5900101E08E048F05FF1279C58C5C7C
:102047008D5D900891E0FEA3E0FFEF2DFDEE3CFCD7
:10205700900891ECF0A3EDF09000EFE0B4021A9035
:102067000893E0FEA3E0FFAA5CAB5DEF2BFBEE3A23
:10207700FA900893EAF0A3EBF08056900101E00490
:10208700C39544854CF0A4FFAEF0900101E08E04A7
:102097008F05FF1279C58C5C8D5D900891E0FEA3DA
:1020A700E0FFEF2DFDEE3CFC900891ECF0A3EDF086
:1020B7009000EFE0B4021A900893E0FEA3E0FFAAB5
:1020C7005CAB5DEF2BFBEE3AFA900893EAF0A3EBDB
:1020D700F00544900101E0C3954450037544009016
:1020E70000AEE05401601B9000A2E0A852B80012B5
:1020F700D39553400DA204B3B35007E560C394CC06
:10210700400280609000A0E075F003A4FFAEF0E508
:10211700412FFF50010E74032FFF50010EE560BEE3
:102127000042D39F403E754501A23440379000A13D
:10213700E075F05EA4FFAEF074058E048F05FF1204
:1021470079C58C5C8D5D12513D900891E0FEA3E04E
:10215700FF9000A1E02FFF50010E900891EEF0A331
:10216700EFF0D234E560C395415002C23485604137
:10217700E5457003022280900102E0C395455003B4
:10218700022272900111E0C39402400302221CE56F
:102197006875F00A84FF7E00900589120048E0F513
:1021A7005B755A00AE5AAF5B9000A1E01279D57407
:1021B700648E048F05FF1279C58C5C8D5D900102DA
:1021C700E004C395458C068D071279D5900102E08E
:1021D7008E048F05FF1279C58C5C8D5D900891E0A8
:1021E700FEA3E0FFEF2DFDEE3CFC900891ECF0A381
:1021F700EDF09000EFE0B4021A900893E0FEA3E040
:10220700FFAA5CAB5DEF2BFBEE3AFA900893EAF07E
:10221700A3EBF08056900102E004C39545854DF08D
:10222700A4FFAEF0900102E08E048F05FF1279C57E
:102237008C5C8D5D900891E0FEA3E0FFEF2DFDEE35
:102247003CFC900891ECF0A3EDF09000EFE0B402B5
:102257001A900893E0FEA3E0FFAA5CAB5DEF2BFBAF
:10226700EE3AFA900893EAF0A3EBF00545900102E5
:10227700E0C395455003754500900891E0FEA3E043
:10228700FF9000B3E0BE00039F500D9000B3E090B5
:102297000891F8E4F0E8A3F09000EFE0B4021290A0
:1022A7000893E0FEA3E0FF9000B3E0BE00059F4067
:1022B70002800D9000B3E0900893F8E4F0E8A3F0F3
:1022C700229000EFE0B401028003022416A204B3B7
:1022D70050030223FD9000BAE0B4017A900891E020
:1022E700FEA3E0FFAC52AD53120003743C8E048F83
:1022F70005FF1279C59000CAE0BC00159D401290F9
:102307000891E0FEA3E0FF9000CCE0BE00039F50E1
:1023170002D203900891E0FEA3E0FFAC52AD531246
:102327000003743C8E048F05FF1279C59000CAE044
:10233700C3940ABC001AD39D4016900891E0FEA3EF
:10234700E0FF9000CCE0C39405BE0004D39F500289
:102357008002C203807A900891E0FEA3E0FFAC52AE
:10236700AD5312000374788E048F05FF1279C59060
:1023770000CAE0BC00159D4012900891E0FEA3E062
:10238700FF9000CCE0BE00039F5004D20380419031
:102397000891E0FEA3E0FFAC52AD5312000374783E
:1023A7008E048F05FF1279C59000CAE0C3940ABC5A
:1023B700001AD39D4016900891E0FEA3E0FF90001D
:1023C700CCE0C39405BE0004D39F50028002C20331
:1023D700A203B34021900891E0FEA3E0FF9000CB59
:1023E700E01279D574648E048F05FF1279C59008C1
:1023F70091ECF0A3EDF0A203B3400CA238400674B1
:1024070024900054F0D238A2034002C2388002C29E
:102417000390004FE06006A204B3B3400280199016
:102427000891E0FEA3E0FF90004FE02FFF50010E60
:10243700900891EEF0A3EFF0A201B34006A202B319
:10244700B3500990001AE4F0A3F0802D900891E0B2
:10245700FEA3E0FF7400D39F74019E401190089182
:10246700E0F8A3E090001AC8F0A3C8F0800B74FF4F
:1024770090001AF8E4F0E8A3F09000D1E0C39404C8
:10248700400C9008F3E0C3940240030225709000CB
:10249700BAE0B40147900891E0FEA3E0FF745E1232
:1024A70079D574058E048F05FF1279C5900891ECD4
:1024B700F0A3EDF09000EFE0B4021F900893E0FE68
:1024C700A3E0FF745E1279D574058E048F05FF12A1
:1024D70079C5900893ECF0A3EDF08045900891E062
:1024E700FEA3E0FF745E1279D5740A8E048F05FF90
:1024F7001279C5900891ECF0A3EDF09000EFE0B4ED
:10250700021F900893E0FEA3E0FF745E1279D57472
:102517000A8E048F05FF1279C5900893ECF0A3ED9E
:10252700F0900891E0FEA3E0FF7402BE000CD39F79
:102537004008752A02752900800A900891E0F5295C
:10254700A3E0F52A900893E0FEA3E0FF7402BE0023
:102557000CD39F4008752E02752D00800A900893B2
:10256700E0F52DA3E0F52E8046900891E0FEA3E06C
:10257700FF7401BE000CD39F4008752A017529001E
:10258700800A900891E0F529A3E0F52A900893E0E6
:10259700FEA3E0FF7401BE000CD39F4008752E0117
:1025A700752D00800A900893E0F52DA3E0F52E9095
:1025B7000018E529F0A3E52AF0A23BB34009C201C0
:1025C70090001AE4F0A3F022900053E090038912E0
:1025D7007A06E0F542754364900053E0FE9000C52B
:1025E700E0D39E4037E56075F00884FF7E008F38A2
:1025F700E56075F00884ADF07C008D3B754008758B
:102607005A03755B96E538C3941F500512118880ED
:102617000690043EE0F5388538438035E56075F06F
:102627000884FF7E008F38E56075F00884ADF07C84
:10263700008D3B754008755A03755BB6E538C39442
:102647001F5005121188800690045EE0F538853822
:1026570043229000FBE0F53D754011755A04755B08
:1026670000AE52AF53E53D75F00FA4FDACF0EDD3CE
:102677009FEC9E4021E53D8E048F05FF1279C5ED45
:1026870075F010A4FFAEF0E56075F01184FD7C00D5
:10269700ED2FF53E800EE56075F01184FF7E00EFAB
:1026A70024F0F53E853E38E56075F01184AFF07E85
:1026B700008F3B12118885383FAE52AF539000FB15
:1026C700E075F00FA4FDACF0EDD39FEC9E402875AC
:1026D7005A04755B10853E38121188853F39853855
:1026E7003AAE52AF53E53D8E048F05FF1279F08D58
:1026F7003B853D3C121202853842754364229000A7
:10270700FBE0F53D754011755A04755B00AE52AF9D
:1027170053E53D75F00FA4FDACF0EDD39FEC9E4063
:1027270021E53D8E048F05FF1279C5ED75F010A4E4
:10273700FFAEF0E56275F01184FD7C00ED2FF53EEC
:10274700800EE56275F01184FF7E00EF24F0F53E00
:10275700853E38E56275F01184AFF07E008F3B123D
:10276700118885383FAE52AF539000FBE075F00FEC
:10277700A4FDACF0EDD39FEC9E4028755A04755B21
:1027870010853E38121188853F3985383AAE52AFE9
:1027970053E53D8E048F05FF1279F08D3B853D3C57
:1027A7001212028538427543649000F6E0B404794A
:1027B700900053E0FE9000C5E0D39E4037E560757A
:1027C700F00884FF7E008F38E56075F00884ADF06F
:1027D7007C008D3B754008755A03755B96E538C3D9
:1027E700941F5005121188800690043EE0F5388545
:1027F70038438035E56075F00884FF7E008F38E543
:102807006075F00884ADF07C008D3B754008755A03
:1028170003755BB6E538C3941F500512118880060F
:1028270090045EE0F5388538432290008FE0B401CC
:102837003BE56875F00A84FF7E008F38E56875F020
:102847000A84ADF07C008D3B75400A755A05755BAF
:1028570012E538C39411500512118880069005AC13
:10286700E0F538E5432538C39464F543900090E0DC
:10287700B4013BE56975F00A84FF7E008F38E5698E
:1028870075F00A84ADF07C008D3B75400A755A05DA
:10289700755B7EE538C39411500512118880069048
:1028A7000618E0F538E5432538C39464F543E54257
:1028B7002543F537900097E0B402109008EBE02528
:1028C70037FE9000EBE0F4042EF5379000EEE0D3EE
:1028D70094014040E56CC394E7501D74E7C3956CC1
:1028E700FE9008EDE08E00F5F0E884FF7E008F385B
:1028F700E5372538F537801CE56CC394E7FE90086B
:10290700EDE08E00F5F0E884FF7E008F38E537C3F1
:102917009538F537A2044006E5422464F537E537D4
:10292700D394644009E537C39464F537800375375A
:10293700009000C7E0C3953750069000C7E0F53711
:1029470022D201900077E0A852B800049553503E78
:10295700900077E0A852B800049553500375370FDD
:10296700900077E004A852B80004955350037537D8
:1029770007900077E02402A852B80004955350024C
:10298700C201900077E060067409900054F0C233EA
:102997007E017F009000CDE01279D59000DCE08EBB
:1029A700048F05FF1279C5E560BC000CD39D400874
:1029B700D23B740A900054F090008FE0B401099064
:1029C70000CEE0C39568400280159000E0E0A85271
:1029D700B8000495535002C201740B900054F09054
:1029E700008FE0B40107E568C394644002801D903E
:1029F7000126E0600D900126E0A852B80006955325
:102A070040028008C201740B900054F0A2014003F9
:102A1700753700C23A90010FE0B40114900110E03D
:102A2700A852B8000495535007E560C3956140026A
:102A3700802A9000B8E0D3941D400B9000B8E0C303
:102A4700941EF5378003753700A237400874159038
:102A57000054F0D23AD237D235022B42C235C237B0
:102A6700900097E0B40306A22DB3B34003022B42B4
:102A77009008EFE0C39405A852B800049553500698
:102A87009008F6E06002801F9000B8E0D3941D40E4
:102A97000B9000B8E0C3941EF537800375370074B8
:102AA7000C900054F0D23A9008EFE0A852B8000416
:102AB700955350069008F6E07002801F9000B8E02A
:102AC700D3941D400B9000B8E0C3941EF5378003E4
:102AD700753700740C900054F0D23A9008EFE0A8D4
:102AE70052B80004955350319000D6E0B40228D272
:102AF700339008F5E0FE9008F6E0D39E5006900864
:102B0700F6E0700280099008F5E4F0C23380069081
:102B170008F5E004F08002C2019008EFE02405A860
:102B270052B80004955350139000D6E0B4020A90AF
:102B370008F6E07002D2338002C201A232B3402706
:102B47009000B8E0D3941D400B9000B8E0C3941EEA
:102B5700F5378003753700A236400674109000548D
:102B6700F0D236D23A8002C23685376D9000B8E08F
:102B7700D3941D4018900086E02537FE900053E05F
:102B870075F01E84FC7F00EE2CF5378029A23AB33E
:102B97004008900086E0F537801C900088E02537D4
:102BA700FE900086E02EFE900053E075F01E84FC38
:102BB7007F00EE2CF537A23BB34005D233756D008D
:102BC70022900053E075F00584FF7E008F38900057
:102BD70053E075F00584ADF07C008D3B75400575BD
:102BE7005A03755BD69000DAE01475F00584FF7E12
:102BF70000E538BE00039F5005121188800BE538A9
:102C070090045F127A06E0F538E5389008EEF09008
:102C170008EEE0FE9000C9E0C39E50089000C9E0AE
:102C27009008EEF09000B8E0D3941D401E9008EE97
:102C3700E0FE900086E02EFE900053E075F01E84C3
:102C4700FC7F00EE2C9008EEF08031A23AB3400AE8
:102C5700900086E09008EEF080229008EEE0FE906B
:102C67000088E02EFE900086E02EFE900053E0756F
:102C7700F01E84FC7F00EE2C9008EEF02290008F6F
:102C8700E0B40136E56875F00A84FF7E0090058997
:102C9700120048E0F547E547D394644010E547C381
:102CA700946475F00F84FF7E008F4780037547009B
:102CB7009000ACE02547F54780069000ACE0F5476B
:102CC70022E56875F00A84FF7E00900589120048A6
:102CD700E0C394694007E568D3946440559000F6D3
:102CE700E0C39403502690088BE0FEA3E0FF740432
:102CF700120039E5601279D5740F8E048F05FF1223
:102D070079C5900889ECF0A3EDF0802490088BE05A
:102D1700FEA3E0FF7404120039E5621279D5740F3F
:102D27008E048F05FF1279C5900889ECF0A3EDF0AA
:102D3700800F90088BE0F8A3E0900889C8F0A3C83B
:102D4700F0A204401A90088BE0FEA3E0FF74031280
:102D570079D57401120039900889EEF0A3EFF0904D
:102D6700009FE0B40262E56BC3944175F00584FFF0
:102D77007E008F38E56B75F00584ADF07C008D3BE8
:102D8700754005755A06755B14E538C394175005E9
:102D970012118880069006B0E0F538900889E0FEA9
:102DA700A3E0FF740A8E048F05FF1279C5E5388CFE
:102DB700068D071279D5740A8E048F05FF1279C51F
:102DC700900889ECF0A3EDF0900889E0FEA3E0FFFE
:102DD70090088FE0FCA3E0FDEDD39FEC9E400F90A1
:102DE700088FE0F8A3E0900889C8F0A3C8F022E5AF
:102DF7000875F004A4FFAEF09006CC120048E090EE
:102E07003C4BF8282873804C85537480479000DC2E
:102E1700E08560F0A4FFAEF074081200398F74806B
:102E270033856274802E856874802985697480244F
:102E3700856A74801F856B74801A856C748015850C
:102E470067748010856674800B856D7480069000AA
:042E57001BE0F57413
:103C4B00022E0D022E0F022E14022E28022E2D02F2
:103C5B002E32022E37022E3C022E41022E46022E0F
:073C6B004B022E50022E5502
:102E5B00E50875F004A4FFAEF09006CD120048E52E
:102E6B000875F004A4FFAEF0E0FC9006CE1200480B
:102E7B00ECFEE0FFEEC39F4003022F63E50875F005
:102E8B0004A4FFAEF09006CC120048E0B40441E578
:102E9B000875F004A4FFAEF09006CE120048E0C314
:102EAB009574500AE508F50CD3923C123FAAE5083D
:102EBB0075F004A4FFAEF09006CD120048E0D39558
:102ECB0074400AE508F50CC3923C123FAA022F612D
:102EDB00E50875F004A4FFAEF09006CD120048E0B3
:102EEB00C395745015E50875F004A4FFAEF0900679
:102EFB00CE120048E0D395745002800AE508F50C19
:102F0B00D3923C123FAAE50875F004A4FFAEF090F3
:102F1B0006CD120048E0D395745015E50875F00402
:102F2B00A4FFAEF09006CE120048E0C39574500A91
:102F3B00E508F50CC3923C123FAA9006D4E0B4010D
:102F4B00099000E8E0D395625002800A7402F50CF8
:102F5B00C3923C123FAA806AE50875F004A4FFAE49
:102F6B00F09006CD120048E0D395744015E5087536
:102F7B00F004A4FFAEF09006CE120048E0C39574A7
:102F8B004002800AE508F50CC3923C123FAAE50803
:102F9B0075F004A4FFAEF09006CD120048E0C39587
:102FAB00744015E50875F004A4FFAEF09006CE1240
:102FBB000048E0D39574400AE508F50CD3923C1217
:102FCB003FAA22AE2FAF3074C9BE000CD39F40086E
:102FDB00782F127A280230E8753001752F00AE5227
:102FEB00AF53E547BE000DD39F40099000BEE0D321
:102FFB00954840028023754800E547C39553F57407
:10300B009000C1E0D395464008E5462574F546800F
:10301B00069000C1E0F5468002054890009AE0D387
:10302B009562401CE560C395614015AE52AF53E508
:10303B0047BE00039F50099000BFE0D39549400263
:10304B00806E9008F0E0A852B800049553500375B9
:10305B004B009008F0E0A852B8000BD395534006F4
:10306B00E5539008F0F0E54B7041E553C39547F5F8
:10307B0074E574D3940540037574059000C0E0C3E8
:10308B0095465007E574C3954640028009E546C353
:10309B009574F54680069000C0E0F5469000C0E0C0
:1030AB00D3954640069000C0E0F546754900800276
:1030BB000549E54B701690009AE0C39562500DE5FB
:1030CB00472405A852B8000695534002800F900084
:1030DB00ADE0F546754B0174789008F0F022AE2FF9
:1030EB00AF3074E9D39F74039E4008782F127A286F
:1030FB0002328F753001752F00754632A22E402A91
:10310B007546199000ADE075F002A4FFAEF0E548EE
:10311B00BE0006D39F4002D22E0548754B03747830
:10312B009008F0F0754A00023276AE52AF53E54785
:10313B006F4E7003023276E547BE000DD39F4009F8
:10314B009000BEE0D395484002800F754800E54BD8
:10315B00C394035003754619800DE547C39553F58A
:10316B0074E5482574F54890009AE0D39562400EBB
:10317B009008F0E0A852B80007D395534002800C9A
:10318B00054A9000ADE0B54A03754B00E54BB4031F
:10319B0006A204B3B34002800A054AE54AB43C03D5
:1031AB00754B02E54BB402299008F0E0A852B80029
:1031BB000ED395534009E5539008F0F0754A0090F3
:1031CB00009AE0C395625009754A0074789008F034
:1031DB00F0E54B705A90009AE0D39562401CE56085
:1031EB00C395614015AE52AF53E547BE00039F50E8
:1031FB00099000BFE0D395494002800875490075DE
:10320B00464B8028E553C39547F574E574D3940575
:10321B00400375740590009AE0D395624008E54928
:10322B002574F5498006E5492406F549754A00E5FC
:10323B004B701690009AE0C39562500DE54724053C
:10324B00A852B80006955340028003754B01E54B1D
:10325B00B40118754619054A9000ADE0B54A0675DC
:10326B004B02754A0074789008F0F0A202B3400349
:10327B00754632E54675F00AA4FFAEF0900895EE60
:10328B00F0A3EFF022E570903C72F8282873023C13
:10329B000B900092E070030235BA9000C8E0B401C5
:1032AB00028003023450900051E0655F6009E553E2
:1032BB004552600302344D7E017F00E5BE1279D585
:1032CB00E5BD2FFF50010E8E5A8F5B9000C6E0B408
:1032DB00461B740E1279D5900076E08E048F05FF95
:1032EB001279C5900899ECF0A3EDF0801DAE5AAFA2
:1032FB005B74101279D5900076E08E048F05FF1267
:10330B0079C5900899ECF0A3EDF0E56C600FE56CD6
:10331B00C394FE50089000EEE0640260028064905B
:10332B0000DCE0B40B1F900899E0FEA3E0FF74E70C
:10333B001279D5E56C8E048F05FF1279C59008992B
:10334B00ECF0A3EDF09000DCE0D3940B4008900080
:10335B00C4E064046002802B900899E0FEA3E0FFB8
:10336B0090089DE0FCA3E0FDEFD39DEE9C400D1279
:10337B007A20900899EEF0A3EFF08007900899E47B
:10338B00F0A3F0900899E0FEA3E0FFEFD39400EEDA
:10339B0094014008D23B7426900054F0A23BB3B387
:1033AB00502C7E057F009000DCE08E048F05FF1211
:1033BB0079C5900899E0FEA3E0FFEFC39DEE9C401A
:1033CB000FAC52AD53740FBC0004D39D500280025E
:1033DB00C23B900092E0B4022790089BE0FEA3E072
:1033EB00FF900899E0FCA3E0FDEF2DFDEE3CFC7493
:1033FB00018C068D07120039900899EEF0A3EFF0BF
:10340B00900899E0FEA3E0FF90089BE0FCA3E0FD91
:10341B00EDD39FEC9E4004D2318002B231900899DB
:10342B00E0F8A3E090089BC8F0A3C8F09000C4E0BC
:10343B0064016006A231B3B34002800690089AE0A3
:10344B00F5600235B8D2317E017F00E5BE1279D529
:10345B00E5BD2FFF50010E8E5A8F5B9000C6E0B476
:10346B00461B740E1279D5900076E08E048F05FF03
:10347B001279C5900899ECF0A3EDF0801DAE5AAF10
:10348B005B74101279D5900076E08E048F05FF12D5
:10349B0079C5900899ECF0A3EDF0E56C600FE56C45
:1034AB00C394FE50089000EEE064026002806490CA
:1034BB0000DCE0B40B1F900899E0FEA3E0FF74E77B
:1034CB001279D5E56C8E048F05FF1279C59008999A
:1034DB00ECF0A3EDF09000DCE0D3940B40089000EF
:1034EB00C4E064046002802B900899E0FEA3E0FF27
:1034FB0090089DE0FCA3E0FDEFD39DEE9C400D12E8
:10350B007A20900899EEF0A3EFF08007900899E4E9
:10351B00F0A3F0900899E0FEA3E0FFEFD39400EE48
:10352B0094014008D23B7426900054F0A23BB3B3F5
:10353B00502C7E057F009000DCE08E048F05FF127F
:10354B0079C5900899E0FEA3E0FFEFC39DEE9C4088
:10355B000FAC52AD53740FBC0004D39D50028002CC
:10356B00C23B900092E0B4022790089BE0FEA3E0E0
:10357B00FF900899E0FCA3E0FDEF2DFDEE3CFC7401
:10358B00018C068D07120039900899EEF0A3EFF02D
:10359B00900899E0F8A3E090089BC8F0A3C8F090BE
:1035AB0000C4E06401600690089AE0F56080037542
:1035BB00600090008EE0700675700302329075BB50
:1035CB0018023C0B023C0B90008EE0700302374359
:1035DB007E017F00E5BE1279D5E5BD2FFF50010EB0
:1035EB008E5A8F5B9000D4E0B4010F7E0F7FFFAC3F
:1035FB005AAD5B127A208E5A8F5B9000F9E0B402C1
:10360B0045AE5AAF5B900024E0FCA3E0FDEDD39FE9
:10361B00EC9E400A900024E55AF0A3E55BF0AE5A0D
:10362B00AF5B900026E0FCA3E0FDEFD39DEE9C404A
:10363B000A900026E55AF0A3E55BF0AE5AAF5B7437
:10364B00041200398F629000F9E0704CAE5AAF5BF8
:10365B00900024E0FCA3E0FDEFD39DEE9C4009120B
:10366B007A208E5A8F5B8006755B00755A00AE5AB6
:10367B00AF5B74101279D59000F8E08E048F05FFC4
:10368B001279C58C5A8D5B74FFBC0009D39D400524
:10369B00855B6280037562FE9000C4E0B40102801A
:1036AB0003023741A204B3B3500E900098E0A85226
:1036BB00B80005D39553500280719000D5E0856218
:1036CB00F0A4FFAEF074648E048F05FF1279C58CE5
:1036DB005A8D5BE56C6016E56CC394FE500F900041
:1036EB00EEE0B402089000DCE0640B60028017AEE1
:1036FB005AAF5B74E71279D5E56C8E048F05FF1218
:10370B0079C58C5A8D5BAE5AAF5B900899E0FCA3E0
:10371B00E0FDEDD39FEC9E4005855B60800BA231F5
:10372B00B3400690089AE0F560800BA231B34006D7
:10373B0090089AE0F5608003756200900091E0704C
:10374B000675700502329075BB19023C0B023C0BDF
:10375B00900091E070030237FBE55FD3955E400369
:10376B000237F9900022E0FEA3E0FFE566127A181B
:10377B00900022EEF0A3EFF07E017F00E5BE127900
:10378B00D5E5BD2FFF50010E8E5A8F5B9000FEE0EA
:10379B007013740A1279D574518E048F05FF127948
:1037AB00C58D668019AE5AAF5B740A1279D58F043A
:1037BB008E057E017F95CDCCCD1278C38F66E566E5
:1037CB00D394644003756664900022E0FEA3E0FF8F
:1037DB00E5662FFF50010E900022EEF0A3EFF09064
:1037EB000095E0048E048F05FF1279C58D6680036A
:1037FB007566329000E1E0700675700702329075C5
:10380B00BB13023C0B023C0B9000E1E0604A7E01D3
:10381B007F00E5BE1279D5E5BD2FFF50010E8E5A04
:10382B008F5B74041200398F679000E3E08567F0BB
:10383B00A4FDACF07464FF1279C58D679000E2E0D3
:10384B008567F0A4FFAEF074FF8E048F05FF12792D
:10385B00C5ED900075F0800375670090008FE070E8
:10386B000675700902329075BB17023C0B023C0BBC
:10387B0090008FE0B40102800302390F7E017F00BC
:10388B00E5BE1279D5E5BD2FFF50010E8E5A8F5B29
:10389B009008F1E060199008F1E0149073B51200F4
:1038AB008CE493FC740193FDEDC39FEC9E4002806E
:1038BB00069008F1E014F09008F1E0C394B3501DAA
:1038CB00AE5AAF5B9008F1E0049073B512008CE434
:1038DB0093FC740193FDEFC39DEE9C400280069018
:1038EB0008F1E004F09008F1E0FE9000B5E08E00E6
:1038FB0088F0A4FFAEF074648E048F05FF1279C5B7
:10390B008D688003756800900090E0700675700BF1
:10391B0002329075BB16023C0B023C0B900090E000
:10392B00B4010280030239BB7E017F00E5BE127930
:10393B00D5E5BD2FFF50010E8E5A8F5B9008F2E03C
:10394B0060199008F2E01490751F12008CE493FC40
:10395B00740193FDEDC39FEC9E400280069008F22C
:10396B00E014F09008F2E0C394B3501DAE5AAF5B75
:10397B009008F2E00490751F12008CE493FC740124
:10398B0093FDEFC39DEE9C400280069008F2E0048D
:10399B00F09008F2E0FE9000BBE08E0088F0A4FFF0
:1039AB00AEF074648E048F05FF1279C58D698003A8
:1039BB0075690075BB1F023C0B023C0B7E017F003F
:1039CB00E5BE1279D5E5BD2FFF50010E8E5A8F5BE8
:1039DB0074091279D574E68E048F05FF1279C58DA3
:1039EB006B900097E0700675700F02329075BB15E7
:1039FB00023C0B023C0B900097E07003023B527EA3
:103A0B00017F00E5BE1279D5E5BD2FFF50010E8E6B
:103A1B005A8F5B74041200398F6A900097E0B401DF
:103A2B00159000EBE0856AF0A4FFAEF0740712006E
:103A3B0039EF9008ECF0900097E0B402159000EB92
:103A4B00E0856AF0A4FFAEF07407120039EF90081E
:103A5B00EBF0900097E0B403028003023B3590003B
:103A6B00D8E07052E56AC39419500FD22D9000B76D
:103A7B00E09008EFF09008F4E4F0E56AD39464402A
:103A8B0004A22D4002802D9008F4E004F09008F47D
:103A9B00E0FE90012AE0B5060B9008EFE004F090F1
:103AAB0008F4E4F09008EFE06496600690012AE0D9
:103ABB007002C22D80639000B7E070349000EBE091
:103ACB00856AF0A4FFAEF074FF8E048F05FF1279A8
:103ADB00C5ED9008EFF0AE52AF53741EBE0006D387
:103AEB009F4002D22DE562D394E54002C22D80297E
:103AFB00E56AC3940A500DAE52AF53741EBE000458
:103B0B00D39F50028002D22DE562D394E54002C2CE
:103B1B002D9000B7E09008EFF09008EFE0C394050C
:103B2B00500674059008EFF0C232900097E0B40491
:103B3B0014E56AC394195002D232E56AD394324029
:103B4B0002C232C22D8003756A009000EEE070064F
:103B5B0075701102329075BB14023C0B023C0B903A
:103B6B0000EEE07003023BF87E017F00E5BE1279A8
:103B7B00D5E5BD2FFF50010E8E5A8F5B900113E0E0
:103B8B007025EFD39421EE940E4005756CFF8015D4
:103B9B00AE5AAF5B74101279D574E38E048F05FFA8
:103BAB001279C58D6C8027AE5AAF5BEFD39449EE7B
:103BBB0094064005756CFF8015AE5AAF5B741012FE
:103BCB0079D574638E048F05FF1279C58D6CE56C06
:103BDB0075F00BA4FFAEF09000DCE08E048F05FFB8
:103BEB001279C590089DECF0A3EDF08003756C0085
:103BFB00900092E0600575BB1A800375BB188000BE
:103C720002329902329C0235CF0235D20237580203
:103C8200375B02381002381302387802387B023967
:103C9200240239270239C40239C70239FE023A0125
:093CA200023B67023B6A023C0B85
:103C0B00E57075F00284AFF07E00EF4E7002D2ECDF
:033C1B000570220F
:097A06002582F58250020583225D
:0F008C0025E050020583258250020583F582226C
:1079A400EF2F500205832582F582E5833E2EF58371
:0179B40022B0
:107A1800CFC39FFF50011E22C3EF9DFFEE9CFE22A5
:087A28000806B6000218062250
:0D79E300A3E004F070061279FCE004F0222D
:0E003900048007C3CE13CECF13CFD5E0F6223E
:1078C300BC000FBE0008ED8FF084FFADF022E4FE94
:1078D300FF22BE000DEF60FE54F0606F20E703024D
:1078E3007979EAC0E0EBC0E078017A0075F001EE47
:1078F30020E710EF25E0FFEE33FE0AC5F023C5F0C5
:1079030030E7F0EA5407F9096A7A007B006001085E
:10791300C3EC9E40167004ED9F4010ED9FFDEC9E5E
:10792300FCE5F0CA4ACA03F5F08005E5F003F5F07B
:10793300C3EE13FEEF13FFD9D77908CACBCAD8D049
:10794300EAFEEBFFD0E0FBD0E0FA22EC8FF084FC00
:10795300ED54F045F0C48FF084FEEDC454F045F0CF
:10796300C48FF084FDEEC4FE54F02DFFEE540F3CA3
:10797300FEADF07C0022790078008FF0EC7E0820C9
:10798300E70DC3CD33CD33C933C9C833C8DEF08463
:1079930049F9E5F08FF0BE00E6FD7C00E9FFE8FE63
:0179A30022C1
:0E79D500F88FF0A4FFE5F0CE88F0A42EFE227D
:10000300EF8DF0A4F9A8F0EF8CF0A428F8EE8DF0B2
:06001300A428FEE9FF2213
:1079B500600D782B0279BF007830D8FED5E0F8222B
:1079C500EEC0E07E001278C3EFFDEEFCD0E0FE22B3
:0C79F000EEC0E07E001278C3D0E0FE2262
:03001B0002001EC2
:0300530002005652
:03009B00020071EF
:03000000027A0F72
:097A0F0075817675D00002530068
:0B004800E5822FF582E5833EF5832260
:0A79FC000582D58202158315822250
:10001E00C0E0C0F0C083C082C0D075D000125203C1
:0B002E00D0D0D082D083D0F0D0E032E0
:10005600C0E0C0F0C083C082C0D075D00012520686
:10006600D0D0D082D083D0F0D0E032C0E0C0F0C093
:1000760083C082C0D075D000125264D0D0D082D056
:0600860083D0F0D0E0324F
:00000001FF
